:100000000C9449180C947A180C947A180C947A1859
:100010000C947A180C947A180C947A180C947A1818
:100020000C947A180C947A180C947A180C947A1808
:100030000C9495200C947A180C947A180C947A18D5
:100040000C947A180C947A180C947A180C947A18E8
:100050000C947A180C947A180C947A180C94F03E3C
:100060000C947A180C944E330C9425330C947A1813
:100070000C947A180C947A180C947A180C947A18B8
:100080000C947A180C947A180C947A180C947A18A8
:100090000C947A180C947A180C947A180C94843373
:1000A0000C947A180C947A180C947A180C947A1888
:1000B0000C947A180C947A180C947A180C947A1878
:1000C0000C947A180C947A180C947A180C947A1868
:1000D0000C947A180C947A180C947A180C947A1858
:1000E0000C947A18114113411541174119411B41D4
:1000F0001D41294145444A444F4459446344DC442A
:100100006D4475447D44874491449B44AA44B4445F
:10011000DC44BE44C844D2449022962299229F22B5
:10012000AA22B222B522BF22293C2C3C1B3C1F3CF8
:10013000253C633C303C343C3A3C3E3C423C483CF1
:100140004C3C503C633C563C5A3C5E3C00407A1070
:10015000F35A00A0724E18090010A5D4E80000E878
:100160007648170000E40B54020000CA9A3B0000D6
:1001700000E1F505000080969800000040420F0065
:100180000000A08601000000102700000000E80326
:10019000000000006400000000000A0000000000F1
:1001A0000100000000002C76D888DC674F0823DFB0
:1001B000C1DFAE59E1B1B796E5E3E453C63AE65183
:1001C000997696E8E6C28426EB898C9B62ED407CAA
:1001D0006FFCEFBC9C9F40F2BAA56FA5F490055A46
:1001E0002AF75C936B6CF9676DC11BFCE0E40D476B
:1001F000FEF520E6B500D0ED902E0300943577058E
:100200000080841E080000204E0A000000C80C3345
:100210003333330F986E12831141EF8D2114893BD4
:10022000E65516CFFEE6DB18D1844B381BF77C1D54
:10023000901DA4BBE424203284725E228100C9F1A7
:1002400024ECA1E53D2715EF03038002CF0300C195
:1002500030ED0464031281E803850078CB05392C66
:10026000003402F70120EA020000C00123C101109E
:10027000C5023E28C701863601483A0155B1020041
:1002800018B603088227F20100260101E00F0F31A2
:100290002B0C0E084EF1370710030E0900E10F007A
:1002A0000E1403110731C148080F0C31360F1180AD
:1002B0007829007F1F8207840684068407827F18BE
:1002C0008207840684068407827F20278E0F900D84
:1002D000920D9001800881018E01820683108404B2
:1002E000850E8504850E8504850E8504850E85049E
:1002F000850E8504850E8504850E8504850E85048E
:10030000850E8504850E8504850E8504850E85047D
:10031000850E85048410840482028E028204800289
:10032000920280069609940C9002811B831985190C
:1003300085198519851985198519851985198519CD
:100340008519851985198519851A830B8E01810BED
:10035000900D920D900F8E28278E0F900D920D907C
:1003600001800881018E01820683108404850E8538
:1003700004850E8504850E8504850E8504850E850D
:1003800004850E8504850E8504850E8504850E85FD
:1003900004850E8504850E8504850E8504850E85ED
:1003A000048410840482028E0282048002920280FD
:1003B00006960680019407820190028104841183CD
:1003C00004850E8504850E8504850E8504850E85BD
:1003D00004850E8504850E8504850E8504850E85AD
:1003E00004850E8504850E8504850E8504850E859D
:1003F00004850E8504850E85058310830781018E93
:1004000001810B900D920D900F8E28278E0F900D6D
:10041000920D9001800C8E01821B8419851985191B
:1004200085198519851985198519851985198519DC
:1004300085198519851A841C821E805D811B83198C
:1004400085198519851985198519851985198519BC
:1004500085198519851985198519851A831C817F48
:1004600024278E0F900D920D900B81018E0B831A15
:10047000851985198519851985198519851985198C
:1004800085198519851985198519841A82028E0A9C
:100490008002920A960680019407820190028104EC
:1004A00084118304850E8504850E8504850E8504DC
:1004B000850E8504850E8504850E8504850E8504CC
:1004C000850E8504850E8504850E8504850E8504BC
:1004D000850E8504850E8504850E850583108307AA
:1004E00081018E01810B900D920D900F8E28278E29
:1004F0000F900D920D900B81018E0B831A8519853B
:1005000019851985198519851985198519851985FB
:1005100019851985198519841A82028E0A8002921A
:100520000A9609940C9002811B83198519851985F7
:1005300019851985198519851985198519851985CB
:100540001985198519851A830B8E01810B900D92DF
:100550000D900F8E287F19800881128206831084E7
:1005600004850E8504850E8504850E8504850E851B
:1005700004850E8504850E8504850E8504850E850B
:1005800004850E8504850E8504850E8504850E85FB
:1005900004850E85048410840482028E0282048005
:1005A00002920280069609940C9002811B831985A1
:1005B000198519851985198519851985198519854B
:1005C000198519851985198519851A831C817F2438
:1005D000278E0F900D920D9001800C8E01821B844E
:1005E000198519851985198519851985198519851B
:1005F000198519851985198519851A840A8E02822B
:1006000008920280069609940C9002811B8319853A
:1006100019851985198519851985198519851985EA
:10062000198519851985198519851A830B8E0181FC
:100630000B900D920D900F8E28278E0F900D920D1E
:100640009001800C8E01821B8419851985198519EA
:1006500085198519851985198519851985198519AA
:100660008519851A840A8E028208920280069606EF
:100670008001940782019009841A851985198519CA
:10068000851985198519851985198519851985197A
:1006900085198519851A831C81018E0F900D920D85
:1006A000900F8E287F19801D821B8419851985194A
:1006B000851985198519851985198519851985194A
:1006C00085198519851B831D811E805D811B8319FA
:1006D000851985198519851985198519851985192A
:1006E00085198519851985198519851A831C817FB6
:1006F00024278E0F900D920D9001800881018E01AC
:10070000820683108404850E8504850E8504850E7B
:100710008504850E8504850E8504850E8504850E69
:100720008504850E8504850E8504850E8504850E59
:100730008504850E8504850E850484108404821446
:10074000820480188024801E821581048411830411
:10075000850E8504850E8504850E8504850E850429
:10076000850E8504850E8504850E8504850E850419
:10077000850E8504850E8504850E8504850E850409
:10078000850E8504850E85058310830781018E0102
:10079000810B900D920D900F8E287F7F7F7B8207BB
:1007A00084068406840782107F7F7F7F3F7F7F10CF
:1007B000860C83028B0983018D0883008F078805CF
:1007C000860686098406850B8405840D8305840DC1
:1007D0008305840D8404830F8304830F8304830FB4
:1007E0008304830F8304830F8304830F8304830FA5
:1007F0008304830F8304830E8404840D8305840C97
:100800008405850B84058609840688058606830091
:100810008F0783018D0883028B098304860C83185C
:1008200083188318831883188318831883188318F0
:1008300083327F7F7F058607860A830289048A08C0
:1008400083008C028C0783008D008E068705890546
:100850008406850886088405840A840A8305840A38
:10086000840A8305830B830B8305830B830B83052A
:10087000830B830B8305830B830B8305830B830B14
:100880008305830B830B8305830B830B8305830B0A
:10089000830B8305830B830B8305830B830B8305FA
:1008A000830B830B8305830B830B8305830B830BE4
:1008B0008305830B830B8305830B830B8305830BDA
:1008C000830B8305830B830B8305830B830B8305CA
:1008D000830B830B837F7F7F7A7F7B880F8D0A90CA
:1008E00009910785068506840A8405830C830583A0
:1008F0000C8305830C83168315840E8B0990079255
:10090000068D01830588078305840B8304840C838B
:1009100004830D8304830D8304830C8404830B857B
:10092000048409860584068A038F0184048D028469
:10093000058A058307867F7F357F1A8409840984A9
:10094000098409847F3D8409840984098409847F9A
:100950007422880F8C0C8F099107860586058509FE
:100960008405840B8404830D8303840D8303830F28
:100970008302830F8302830F8302830F8302830F1B
:100980008302840D8403830D8403840B850484090E
:1009900086048605880594068E0083078B02830AE9
:1009A00086048316831583168303830E8303830DC6
:1009B0008403840C8305830B8405840985068505DF
:1009C0008608900A8E0C8B11867F7F332485118BCD
:1009D0000C8F0991078605860684098405840B849B
:1009E00004840B8404830D8304830D8304830D83AB
:1009F00004840B8405830B8306840984078505859D
:100A0000098F0B8D0B8F09910785078505840B8452
:100A100004830D8303840D8402830F8302830F8379
:100A200002830F8302830F8302830F8302840D846A
:100A300002840D8403840B84048607860593079142
:100A4000098F0D897F7F313796039603960396169B
:100A500083158315831583158414841484158315D5
:100A600084148415841484158315841583158415C2
:100A700084158315841583168315841583168316B0
:100A800083168315841583168316837F7F532486EC
:100A9000118B0C8E0A9008860585068509840584CD
:100AA0000B8305830C8403840D8303830E830383EC
:100AB00016831583168304860A83028B0783008EB0
:100AC0000694058805860486098404850B840384BE
:100AD0000D8303840D8402830F8302830F830283BB
:100AE0000F8302830F8302830F8303830D840383A9
:100AF0000D8304840B84058409850586058607918A
:100B0000098F0C8C0F887F7F313A910891089108EA
:100B1000910882168316831683168217821782160F
:100B20008302870B83008B0991089207860586064E
:100B300084098505830B8416831684168316831611
:100B4000831683168303830E8303830D8403830D2F
:100B50008304840B8405840985058605860791092D
:100B60008F0B8D0F877F7F32458315841485138605
:100B700013861287118300831183008310830183FE
:100B80000F8302830E8402830E8303830D83048309
:100B90000C8305830B8405830B8306830A830783F9
:100BA00009840783098308830883098307830A83E9
:100BB000079702970297029711831683168316836D
:100BC000168316831683168316837F7F4A23870F27
:100BD0008D0B900891078605860684098405840B91
:100BE0008404840B8404830D8304830D8304830DA8
:100BF0008315841584148414850D8B0E89108B0E37
:100C00008C148615841684158402830F8302830F47
:100C10008302830F8302840D8402840C8503840B7A
:100C20008404850985058605860791098F0B8D0F3C
:100C3000877F7F4D2487108C0B8F0991088505864F
:100C40000684098406840A8306830B8404840C8347
:100C500004830D8304830D8304830D83168315841D
:100C600015841484148513851286118710881088C2
:100C70000F881087118612851385148414841583B8
:100C8000168315960396039603967F7F4529821750
:100C900082168316831584148512870D8C0D8C0D96
:100CA0008700830D840383168316831683168316A9
:100CB000831683168316831683168316831683166C
:100CC000831683168316831683168316831683165C
:100CD000831683168316837F7F4C23870F8D0B8F9C
:100CE0000991078605860684098406830B8305849B
:100CF0000B8404830D8304830D8304830D8303839A
:100D00000F8302830F8302830F8302830F83028387
:100D10000F8302830F8302830F8302830F83028377
:100D20000F8302830F8302830F8302830F83028367
:100D30000F8302830F8303830D8304830D83048356
:100D40000D8304840B8405830B8306840984068643
:100D500005860791098F0B8D0F877F7F327F7F7FFD
:100D6000558409840984098409847F387F7F458AF2
:100D7000058A058A058A7F7F7F2B7F7F7F7F3F19CA
:100D8000118309810181078103820380008006812C
:100D90000181008007837F7F2C01830A820A810AF8
:100DA000810A810A810A810A810A810A810A810BEA
:100DB000810B82088109810A810A810A810A810ADC
:100DC000810A810A810A81098207831304810A81C9
:100DD0000A810A810A810A810A810A810A810A81BB
:100DE0000A810A810A810A810A810A810A810A81AB
:100DF0000A810A810A810A810A810A810A8112060E
:100E000083078209810A810A810A810A810A810A8B
:100E1000810A810A81098108820B810B810A810A7A
:100E2000810A810A810A810A810A810A810A820A69
:100E3000830E488901890882078207820782088118
:100E4000088207820782078208890189544D820639
:100E5000820081068101810681028104810381046F
:100E6000810381048104810281058102810581025F
:100E70008106810081078100810781008108820944
:100E80008209820981098206840783144E810681C2
:100E90000182048202810481048102810582008230
:100EA000068408820884068200820581028104810A
:100EB000048102820482018106815B6B81048204C9
:100EC000810081048204810081048000800481010A
:100ED00081028100810281028102810081028102FE
:100EE00081028100810281028102800280028103ED
:100EF00081008102810081048100810281008104DE
:100F000081008102810081058204820682048206BA
:100F10008204827F0147810681008106810181046C
:100F200081028104810281048103810281048102A2
:100F30008104810281058100810681008106840788
:100F400082088258558106810281068102810681CC
:100F50000281068102810681028106810281068169
:100F60000281068102810681028105820282038359
:100F70000386008104840181620F8104810481045D
:100F80008102850085028104810481048104810439
:100F90008104810481048104830382314A840587AA
:100FA000028203810281058101810A840786078408
:100FB00009810181058101820382028704855631FE
:100FC00081008201850182048105810581058105F9
:100FD00081058105810581058105813B5E83018154
:100FE00004860081038301840381058202820681D5
:100FF00002810781028107810281078102820681C5
:1010000003810582038301840486008106830181B4
:101010000C810C810C810C810C811F5B810183068A
:101020008100860484018303820581038106820294
:101030008107810281078102810781028106820284
:101040008205810384018303810086048101830674
:10105000810C810C810C810C81285E8407880483BB
:101060000283038106810282068201810881018157
:101070000881018108810182068202810681038341
:101080000283048807846D5B8101840581008604E6
:101090008303820382058103810681038106810324
:1010A0008106810381068103810681038106810314
:1010B00081068103810681038106816A7F058101A2
:1010C00083038305810085008604830284028203F2
:1010D00082048204810381058105810381058105E4
:1010E00081038105810581038105810581038105D6
:1010F00081058103810581058103810581058103C6
:1011000081058105810381058105817F1B0781039D
:1011100081038103810381038103810381038103AF
:10112000810381038103810381038103810381039F
:10113000812B198109810981098109810482018139
:10114000038202810282038101820481008205857B
:101150000586048201810481028203810381038167
:101160000382028104810281048253078103810387
:10117000810F810381038103810381038103810343
:10118000810381038103810381038103810381033F
:1011900081038101830182080781038103810F811B
:1011A000038103810381038103810381038103811F
:1011B00003810381038103812B10810C810C810C3D
:1011C000810C810C810184058100860483038203E4
:1011D00082058103810681038106810381068103E3
:1011E00081068103810681038106810381068103D3
:1011F000810681038106816A5E8301810486008104
:1012000003830184038105820281078102810781B2
:1012100002810781028107810282068103810582A2
:101220000383018404860081068301810C8102818D
:101230000781028106820382038204890685130ADC
:10124000830284028105810581038600860281056F
:10125000810581058105810581058105810581055E
:101260008105813B588307870483018303810581BE
:1012700002820681018B018B01810B820B81058229
:1012800002830183048707836619810C810C810C1A
:10129000810C81068301810486008103830184031C
:1012A0008105820282068102810781028107810213
:1012B0008107810282068103810582038301840400
:1012C000860081068301816A528306870383018237
:1012D00003810581018209810A810A810A820581CF
:1012E0000281058102830182048706835E10810CDE
:1012F000810C810C810C810C8101830681008604A4
:1013000084018303820581038106820281078102B1
:1013100081078102810781028106820282058103A1
:1013200084018303810086048101836D57850588CC
:1013300004810482038105810B8105870389028270
:101340000581028106810281068102820383038670
:10135000008302840282610B830385018201820083
:101360008103810081038100820182018503837FE3
:101370001A7F7F1D8C2610820781008105810281E2
:1013800003810481018106817F6F098403840681C2
:101390000681068106810681068106810681068115
:1013A0000681068106810681068106810681068105
:1013B00006810681038403841401800B800B810B5A
:1013C000800B800B810B800B800B810B800B800BC3
:1013D000810B800B800B810B800B800B810B800BB2
:1013E000800B810B800B800B810B800E0B840384A0
:1013F00003810681068106810681068106810681B8
:1014000006810681068106810681068106810681A4
:101410000681068106810684038412118C028C0CDD
:10142000820B820B820C810C810C820B820B820C52
:10143000810C810C820B820B820B820C8D018D70D2
:101440000F8209820082078202810781038205825E
:10145000048105810681038107820182088101815F
:101460000A830B830C810D810D810D810D810D810E
:101470000D810D81760F810881018206820281062D
:101480008104810481058202820681028108810033
:101490008109840A820B820A810081088200820706
:1014A0008102810681048104820482038106810213
:1014B0008206820082088268168206820682008185
:1014C00006820681018106820681018204810081F3
:1014D00004820281048100810481038104810081EE
:1014E00004810381048100810481038202810281DD
:1014F00002820481028102810281058102810281CE
:1015000002810581028102810281058200810481BC
:1015100000820681008104810081078100810481AD
:10152000008107810081048100810783068308828E
:101530000682098206827F250E8208820081088148
:101540000181088101810881028106810381068170
:101550000381068104810481058104810581048160
:101560000681028107810281078102810881008151
:101570000981008109840A820B826E13810981032B
:101580008109810381098103810981038109810323
:101590008109810381098103810981038109810313
:1015A0008109810381098103810981038109810303
:1015B0008109810382078204820582068908877F68
:1015C000020D9B05810B810B810B810B810B810B24
:1015D000810B810B810B810B810B810B810B810BAB
:1015E000810B816714850789048205820381078145
:1015F000038107810381078202820D840B860B859C
:101600000C830D8201820881028108810281088198
:1016100002830582038A068673128B048C03810879
:101620008202810981028109810281098102810985
:101630008102810881038C038B0481078203810866
:101640008103810882028109810281098102810965
:10165000810281098102810981771886098A0683BE
:1016600004830482088203810A8102820A82018142
:101670000C8101810C8101810C8101810C8101812E
:101680000C8101810C810182068002820281058227
:1016900001810382058504830483068C0786018209
:1016A000108073118A048B038107820281088102F2
:1016B00081088102810881028108810281078202FA
:1016C0008B038A04810D810D810D810D810D810DAA
:1016D000810D817B1886098A06830483048208822F
:1016E00003810A8102820A8201810C8101810C81BD
:1016F00001810C8101810C8101810C8101810C81AE
:1017000001820A8202810A8103820882048304839F
:10171000068A09867F0A138208810382088103836F
:101720000781038406810381008106810381008291
:101730000581038101820481038102810481038187
:101740000282038103810382028103810481028179
:101750000381048201810381058200810381068166
:10176000008103810684038107830381088203814A
:1017700008827F16820A8203830883038308830317
:101780008308830381008106810081038100810633
:101790008100810381008106810081038101810430
:1017A000810181038101810481018103810181041F
:1017B0008101810381028102810281038102810210
:1017C0008102810381028102810281038103810000
:1017D00081038103810381008103810381038403E9
:1017E000810381048204810381048204817F140EB9
:1017F000810A810A810A810A810A810A810A810A91
:10180000810A810A810A810A810A810A810A810A80
:101810008A018A5A12810882028107820381068224
:101820000481058205810482068103820781028288
:101830000881018209810083098708830182078268
:101840000382068105810681058205810682048165
:10185000078203810882028109827615810A810A42
:10186000810A810A810A810A810A810A810A810A20
:10187000810A810181068101810681018106810140
:10188000820482028804865E0781038103810381CA
:101890000381038103810381038103810381038128
:1018A0000381038103810381038103812B13810958
:1018B00081038109810381098103810981038109F0
:1018C000810381098103810981038D038D038109CE
:1018D00081038109810381098103810981038109D0
:1018E00081038109810381098103810981038109C0
:1018F000817F1886098A0682058304820881048113
:10190000098202820F81108110810587028105877B
:1019100002810B8102810B8102820A81038109828B
:10192000038207830483048405890081078503807B
:101930007F06108B028B02810C810C810C810C8143
:101940000C810C8A038A03810C810C810C810C812F
:101950000C810C810C8173118C028C02810D810D24
:10196000810D810D810D810D8B038B03810D810D07
:10197000810D810D810D810D8C028C701389078B77
:10198000058106830481088203810981038109821C
:1019900002810A8102810A8102810A8102810A810F
:1019A00002810A8102810A81028109820281098100
:1019B0000381088203810683048B05897F031786D0
:1019C000088A058304830382088103810A810182D6
:1019D0000A8101810F810F810F810F810F810B819E
:1019E00001820A81028109820282088104830483C0
:1019F000058A08867F02128A058C0381078203818B
:101A000008810381088103810881038108810381A2
:101A10000782038A058C0381078203810981028181
:101A20000981028109810281098102810782038C77
:101A3000038A7A15830B830B830A81018109810153
:101A40008109810181088103810781038107810365
:101A50008106810581058105810589048B03810744
:101A60008103810781028109810181098100820945
:101A7000826F21880D82068209820A8107810D8189
:101A800005810F8104800683018003810281048126
:101A90000283038102810381048104810181048125
:101AA0000481048101810381058104810181038115
:101AB0000581048101810381048104810281038104
:101AC00004810481028103810481038104810381F3
:101AD00002820281058104830184078117811781B5
:101AE0000B81098205830D876C10850488038203AE
:101AF00082018205810181068101810681098208B6
:101B00008208820882098109820982238209820966
:101B1000825F62820C820C830C820D8108820783B3
:101B2000078208827F155186018613860186636BC2
:101B30008208820783078208810D820D820C820C45
:101B4000827F0C2B8203820382348203820382050C
:101B500080048104800481172B82038203823482F3
:101B600003820382321F8505880482038202820574
:101B7000810281078101810781018107810182053D
:101B80008202820383028A048401810B810181061F
:101B90008102810681038104820388058665208392
:101BA0000787058103810481058103810581038104
:101BB00005810481038106850687048203820281F0
:101BC00007810181078101810781018107810282EB
:101BD000038203890585651C8B018B0A810A8209B2
:101BE000820A810A820A810A810B810A820A810B98
:101BF000810B810A810B810B816920840688038215
:101C00000481038106810281068101810B810184A7
:101C1000048A028303820282058201810781018195
:101C20000781018107810281058202820382048883
:101C30000585651D89038903810B810B810B81005B
:101C400084058902830382028106820B810B810B4A
:101C50008101810781018205820282038203890555
:101C6000856524810A8209830983088100810781AF
:101C7000018106810281068102810581038104813F
:101C8000048103810581038B018B09810B810B8109
:101C90000B81641F8506870482038203810581020C
:101CA0008205810B810A82078408850B820B8101E2
:101CB00081078101810781018205820282038203FB
:101CC000890585651F850589038203820282068155
:101CD00001810781018107810B810A8208830784C2
:101CE00006840783088209820A810B8B018B62229A
:101CF000810B810A82078507850B810B810B810B84
:101D0000810B810B810B810B810B810B810B810B73
:101D10008166208307870483018303810581028212
:101D2000058201810781018107810181078101818C
:101D3000078101810781018107810181078101827A
:101D40000582028105810383018304870783660D71
:101D50008105810580058105810580058105810555
:101D60008005810581058005810581058005810546
:101D7000810580058105812D71820382038232589D
:101D80008501856871820382038205800481048055
:101D90000481175381078107810487018704810724
:101DA0008107816710810981098106800181018095
:101DB00002890385068306810181048201820480F1
:101DC00003807F36078106800681068006810581B3
:101DD00005810681058105810581058105810581D2
:101DE00005810581058104810581058105800581C5
:101DF000058005810D0D8105800581058005810522
:101E000081058104810581058105810581058105A3
:101E10008105810581058106810581058106800690
:101E20008106800681070682028202820480038185
:101E300002817415840A8608820282078104810760
:101E400081048107810382088101820A840A830B4D
:101E50008503810382018202810282038201810261
:101E6000810584038106830381078104820485033D
:101E700088018203850482762D820781058605808C
:101E80000681028104810581048102810681048129
:101E90000280078104810181088102810280098614
:101EA00001800C82028102820C80018609800281FD
:101EB00002810881018104810780028104810681F9
:101EC00002810481058104810281068005860581E5
:101ED000078207807F0C1F850589038203820281A8
:101EE00007810181078101810B820B810A870781AC
:101EF0000B810B810B810A810B860280018B018192
:101F00000483632E8101810C8002800D8002800C8D
:101F10008101810C8002800D800280088D08800282
:101F2000800D8002800D800280088D088002800D67
:101F30008002800C8101810C8002800D8002800C67
:101F40008101817F0D098001800380018003800170
:101F50008003800180038001800380018003800171
:101F6000807F110A81058105810581058105810533
:101F70008105810581058105810581058115810521
:101F80008105813A7F0100003048483000000000A0
:101F9000000000000000000000324C0000000000C3
:101FA0000000000000000040202020202020102001
:101FB0002020202020400000404040404040404041
:101FC00040404040400000102020202020204020A1
:101FD000202020202010000000000000FC04083019
:101FE0004080FC0000000000000000008484848425
:101FF000844C3404087000000000000088885020E1
:102000005088880000000000000000008282829258
:1020100092AA440000000000000000008282828238
:102020004428100000000000000000008484848424
:10203000844C34000000000000004040E04040407C
:1020400040403000000000000000000070888070F8
:10205000088870000000000000000000B0C8808008
:10206000808080000000000000000000344C848468
:10207000844C34040406000000000000B0C88484CE
:1020800084C8B08080800000000000003844828254
:10209000824438000000000000000000B0C88484C2
:1020A000848484000000000000000000ACD2929202
:1020B000929292000000000000C04040404040402A
:1020C0004040400000000000008080808890A0C058
:1020D000A0908800000000000000100030101010D8
:1020E0001010101090600000000040004040404080
:1020F000404040000000000000808080B0C8848420
:10210000848484000000000000000000304C8484BF
:10211000844C340408700000003048404040E040E7
:10212000404040000000000000000000384484F8F7
:10213000804438000000000000000404344C848413
:10214000844C34000000000000000000384480800F
:10215000804438000000000000008080B0C8848403
:1021600084C8B00000000000000000007008047483
:102170008C8C7400000000000040404020000000F3
:10218000000000000000000000000000000000004F
:1021900000000000FF000000000000000000000040
:1021A00000000000000000102844000000000000B3
:1021B000000000000000000000000000000000001F
:1021C0000000000000000000E0202020202020204F
:1021D000202020E000000000040408081010202047
:1021E0004040808000000000E0808080808080800F
:1021F000808080E00000000000FE02040810102033
:102200004080FE00000000000082828244281010FE
:1022100010101000000000000082824428101028D6
:102220004482820000000000000000008080808066
:102230008080888088804900550055002200220057
:1022400000000000000000000082828282444428D6
:1022500028101000000000000082828282828282A8
:10226000824438000000000000FE10101010101012
:1022700010101000000000000038448280601C0232
:10228000824438000000000000F884828284F890C4
:1022900088848200000000000038448282828282AA
:1022A000824438080600000000F88482828284F8A4
:1022B0008080800000000000003844828282828298
:1022C000824438000000000000C2C2A2A292928A9A
:1022D0008A8686000000000000000000C180C180E6
:1022E000A280A28094809480888088808080808072
:1022F000000000000000000000808080808080805E
:102300008080FC000000000000848890A0C0A090A5
:102310008884820000000000000202020202020221
:10232000824438000000000000E04040404040404F
:102330004040E000000000000084848484FC848429
:102340008484840000000000003C428080809C82E5
:1023500082423C000000000000FE808080F8808007
:10236000808080000000000000FE808080FC808073
:102370008080FE000000000000F884828282828259
:102380008284F80000000000003C42808080808051
:1023900080423C000000000000F8848284F88482BF
:1023A0008284F80000000000001010282844447CBB
:1023B0008282820000000000003C4299A5A5A5A5EC
:1023C0009E403E00000000000038448202040810D5
:1023D00010001000000000000000804020100810D5
:1023E00020408000000000000000000000F800F81D
:1023F00000000000000000000000081020408040A5
:10240000201008000000000000000000C0C000C054
:10241000C04080000000000000000000C0C000C0FC
:10242000C0000000000000000038448282463A02EA
:1024300002047800000000000038448244384482DE
:102440008244380000000000007E020204040808F4
:102450001010100000000000003C408080B8C482D2
:10246000824438000000000000FC808080F80402F4
:10247000028478000000000000040C14244484FE50
:102480000404040000000000007884020438040200
:102490000284780000000000003844820204182002
:1024A0004080FE000000000000103050101010109E
:1024B00010107C00000000000038444482828282B8
:1024C00044443800000000000404080810102020D4
:1024D000404080800000000000000000000000007C
:1024E00000C0C00000000000000000000000F80074
:1024F00000000000000000000000000000000000DC
:1025000000C0C04080000000000000002020F82033
:102510002000000000000000000010925438549287
:1025200010000000000000C020100808040404048B
:102530000408081020C0000C1020404080808080DB
:1025400080404020100C000040404080000000000F
:102550000000000000000000002050888850205239
:102560008C8C7300000000000061919264081026BA
:102570004989860000000000003C424040704070E5
:102580004040FE000000000000242424FF2424FF1B
:102590002424240000000000A0A0A00000000000EF
:1025A000000000000000000000404040404040406B
:1025B000400040000000000000000000000000009B
:1025C0000000000000000C0C0C0C0C0C0C0C0C0C93
:1025D0000C0C0C0C0C0C2020202020202020202073
:1025E0000C0C0C0C0C0C0C0C0C0C0C0C0C0C0C0C2B
:1025F0000C0C0C0C0C0C0C0C0C0C0C0C0C0C0C0C1B
:102600000C0C0C0C0C0C0C0C0C0C0C0C0C0C0C0C0A
:102610000C0C0C0C0C0C0C0C0C0C0C0C0C0C0C0CFA
:102620000C0C0C0C0C0CA807A807A807A807A807F7
:10263000A807A807A807A807A807A807A807A80722
:10264000A8079A07A807F106A4063906D00555057C
:10265000EE0461040B045803CB02B302A807A807D9
:10266000A807A807A807A807A807A807A807A807F2
:10267000A807A807A807A807A807A807A807A807E2
:10268000A807A807A807A807A807A807A807A807D2
:10269000A807A807A807A807A807A807A807A807C2
:1026A000A807A807A807A807A807A807A807A807B2
:1026B000A807A807A807A807A807A807A807A807A2
:1026C000A807A807A807A807A807A807A807A80792
:1026D000A807A807A807A807A807A807A807A80782
:1026E000A807A807A8070C0C0C0C0C0C0C0C0C0C65
:1026F0000C0C0C110F0C1B1B1B1B1B1B1B1B1B1B7C
:102700000F0C0C0C0C0C0C0C0C0C0C0C0C0C0C0C06
:102710000C0C0C0C0C0C0C0C0C0C0C0C0C0C0C0CF9
:102720000C0C0C0C0C0C0C1B0C0C0C0C0C0C0C0CDA
:102730000C0C0C2A0C0C1D0C0C0C0C0C0C0C0C0CAA
:102740000C0C070C0C0C7A0D7A0D7A0D7A0D7A0DA3
:102750007A0D7A0D7A0D7A0D7A0D7A0D7A0D7A0D41
:102760006C0D5D0D7A0DDA0C8D0C340CCD0B680BF5
:10277000090B8E0A470ACC09510939097A0D7A0DDD
:102780007A0D7A0D7A0D7A0D7A0D7A0D7A0D7A0D11
:102790007A0D7A0D7A0D7A0D7A0D7A0D7A0D7A0D01
:1027A0007A0D7A0D7A0D7A0D7A0D7A0D7A0D7A0DF1
:1027B0007A0D7A0D7A0D7A0D7A0D7A0D7A0D7A0DE1
:1027C0007A0D7A0D7A0D7A0DD9087A0D7A0D7A0D77
:1027D0007A0D7A0D7A0D7A0D7A0D7A0D7A0D7A0DC1
:1027E00032087A0D7A0DAD077A0D7A0D7A0D7A0DD1
:1027F0007A0D7A0D7A0D7A0D7A0D7A0D7A0D7A0DA1
:102800007A0D7A0D7A0D050808130E1511060808C1
:102810000C0A070807080E0E0E0E0E0E0E0E0E0EF8
:1028200007070E090E0D1910111212100F131206C0
:102830000D110D151213101311100E120F170F108A
:1028400010090D090C0D090E0F0D0F0E080F0F06C4
:10285000060C06160F0F0F0F080C070E0C120D0DAD
:102860000C0D0D0D0F01841F631F451F031FD61E86
:10287000781E331E261EF51DC41DA41D931D841D28
:102880007F1D781D4F1D121DEF1CC41C931C621C64
:10289000331CFA1BD71B9E1B651B581B431B2F1B8E
:1028A000261B121BE91A721A331AF619BE197C1963
:1028B00057193219F218AD1888185B181418EF1749
:1028C00073171617D416A3165A161916E415C11540
:1028D0007B153815B814751440141B14EC13B91378
:1028E0008A137613711357132C13ED12C812891221
:1028F00064123F12F811B91198116B1132110D11B8
:10290000BC1087105A101B10DC0FBF0F9C0F790FE3
:10291000440F150FBB0E8C0E4D0E320EFF0DCC0D5D
:10292000990D800D7F0D06030409080909030707A7
:102930000806030605070808080808080808080824
:10294000030306060608090808080808080808041A
:102950000808070A0808080808080808080A0808F4
:102960000804070407090407070707070607070401
:1029700005060408070807080606050708080607ED
:10298000070503050806B625A6259625862576257E
:102990006625562546253625262516250625F624A0
:1029A000E624D624C624B624A62496248624762497
:1029B0006624562446243624262416240624F62388
:1029C000E623D623C623B623A6239623862376237F
:1029D0006623562346233623262316230623F62270
:1029E000D622C622B622A6229622862276226622E7
:1029F00056224622262216220622F621E621D6213A
:102A0000C621A6218621762166215621462136211E
:102A1000262116210621F620E620D620C620B62043
:102A2000A620962086207620662056204620362036
:102A3000262016200620F61FE61FD61FC61FB61F2B
:102A4000A61F961F861F00002000230026002900D5
:102A50002C002F00320000010000030106010901D3
:102A60000000000000000000000886292629100050
:102A700000000000662806281A0000000000462713
:102A8000E626302626C62530000000000000002281
:102A900000250028002B002E003100340002010028
:102AA00000050108010B01050505050705080808D3
:102AB00008020202020A0A080804040404010101CF
:102AC00001010101010303030303030303040707D7
:102AD000070C0C0C0C0C0C0C0C0202020206060675
:102AE00006060606060B0B0B0B0B0B0B0B0102105D
:102AF0002020080810204010204080020102010818
:102B000004020101020408102040808040201008C7
:102B10000402018004020180402010080402010820
:102B20000402010102040810204080010204081080
:102B300020408000000000003E5B4F5B3E3E6B4F3C
:102B40006B3E1C3E7C3E1C183C7E3C181C577D573F
:102B50001C1C5E7F5E1C00183C1800FFE7C3E7FFEB
:102B60000018241800FFE7DBE7FF30483A060E267E
:102B700029792926407F050507407F05253F5A3CD6
:102B8000E73C5A7F3E1C1C08081C1C3E7F14227F19
:102B900022145F5F005F5F06097F017F00668995F1
:102BA0006A606060606094A2FFA29408047E0408DA
:102BB00010207E201008082A1C08081C2A08081E5D
:102BC000101010100C1E0C1E0C30383E3830060E43
:102BD0003E0E06000000000000005F00000007003D
:102BE0000700147F147F14242A7F2A1223130864F9
:102BF0006236495620500008070300001C2241009D
:102C00000041221C002A1C7F1C2A08083E080800DC
:102C1000807030000808080808000060600020107C
:102C20000804023E5149453E00427F400072494936
:102C300049462141494D331814127F102745454517
:102C4000393C4A4949314121110907364949493638
:102C5000464949291E0000140000004034000000CD
:102C600008142241141414141400412214080201FF
:102C70005909063E415D594E7C1211127C7F49492B
:102C800049363E414141227F4141413E7F494949C8
:102C9000417F090909013E414151737F0808087FBE
:102CA00000417F41002040413F017F081422417FC5
:102CB000404040407F021C027F7F0408107F3E415D
:102CC00041413E7F090909063E4151215E7F0919B4
:102CD0002946264949493203017F01033F404040CC
:102CE0003F1F2040201F3F4038403F6314081463BB
:102CF00003047804036159494D43007F4141410277
:102D000004081020004141417F04020102044040B8
:102D1000404040000307080020545478407F284476
:102D200044383844444428384444287F3854545460
:102D30001800087E090218A4A49C787F080404786F
:102D400000447D40002040403D007F1028440000AA
:102D5000417F40007C047804787C0804047838447F
:102D6000444438FC1824241818242418FC7C080433
:102D70000408485454542404043F44243C40402054
:102D80007C1C2040201C3C4030403C4428102844FF
:102D90004C9090907C4464544C44000836410000B0
:102DA00000770000004136080002010204023C26C0
:102DB00023263C1EA1A161123A4040207A38545487
:102DC000555921555579412154547841215554780C
:102DD0004020545579400C1E5272123955555559A0
:102DE000395454545939555454580000457C4100C5
:102DF00002457D420001457C40F0292429F0F0285D
:102E00002528F07C545545002054547C547C0A09F4
:102E10007F4932494949323248484832324A484863
:102E2000303A4141217A3A42402078009DA0A07D6D
:102E300039444444393D4040403D3C24FF2424482B
:102E40007E4943662B2FFC2F2BFF0929F620C088D3
:102E50007E090320545479410000447D41304848A4
:102E60004A32384040227A007A0A0A727D0D1931BE
:102E70007D2629292F28262929292630484D40201A
:102E8000380808080808080808382F10C8ACBA2FF6
:102E9000102834FA00007B000008142A142222149F
:102EA0002A1408AA005500AAAA55AA55AA0000008B
:102EB000FF00101010FF00141414FF001010FF008A
:102EC000FF1010F010F0141414FC001414F700FF9D
:102ED0000000FF00FF1414F404FC141417101F105A
:102EE000101F101F1414141F00101010F000000009
:102EF000001F101010101F10101010F01000000014
:102F0000FF101010101010101010FF10000000FF24
:102F1000140000FF00FF00001F10170000FC04F465
:102F200014141710171414F404F40000FF00F7141D
:102F3000141414141414F700F714141417141010A4
:102F40001F101F141414F4141010F010F000001FC0
:102F5000101F0000001F14000000FC140000F010FF
:102F6000F01010FF10FF141414FF141010101F00A5
:102F7000000000F010FFFFFFFFFFF0F0F0F0F0FFA7
:102F8000FFFF0000000000FFFF0F0F0F0F0F38447E
:102F90004438447C2A2A3E147E02020606027E023F
:102FA0007E0263554941633844443C04407E201E00
:102FB0002006027E020299A5E7A5991C2A492A1C2F
:102FC0004C7201724C304A4D4D303048784830BC1C
:102FD000625A463D3E494949007E0101017E2A2A46
:102FE0002A2A2A44445F444440514A444040444AC7
:102FF00051400000FF0103E080FF000008086B6BF8
:10300000083612362436060F090F0600001818007D
:1030100000001010003040FF0101001F01011E00E0
:10302000191D1712003C3C3C3C0000000000000051
:103030002100240027002A002D0030003300010168
:103040000000040107010A0100000A0B02090C0D2F
:103050000E0807030401000000000000000000004B
:103060000000000000000000000000000000000060
:10307000000000001211100000000000000000001D
:1030800000000000000000000000000000003649C1
:103090002A4911241FBECFEFD1E2DEBFCDBF00E031
:1030A0000CBF17E0A0E0B2E0E0E1F5EA00E00BBF02
:1030B00002C007900D92A63AB107D9F72CE0A6EA14
:1030C000B7E001C01D92A331B207E1F718E1C8E4EF
:1030D000D8E100E006C021970109802FFE010E947F
:1030E0003050C734D10780E00807A9F70E943A3F63
:1030F0000C9477520C940000089580E090E00895BD
:10310000CF92DF92EF92FF920F931F93CF93DF93B3
:10311000FC0122812223A9F1EC010E94AC3E6B014B
:103120007C018F819885A985BA850097A105B10595
:1031300009F14B815C816D817E8197018601081BBD
:10314000190B2A0B3B0B041715072607370790F4BA
:10315000C816D906EA06FB06A0F480959095A095BE
:10316000B0958C199D09AE09BF0984179507A6076C
:10317000B70738F0E881F9811995CF82D886E986BA
:10318000FA86DF91CF911F910F91FF90EF90DF9022
:10319000CF9008954F925F926F927F928F929F92FD
:1031A000AF92BF92CF92DF92EF92FF920F931F9355
:1031B000CF93DF93EC014B016A01290158013701DC
:1031C000E12CF12C89019A01AB01BC0180ED98E062
:1031D0000E94E33684E08093F00873019601A40115
:1031E000BE0180ED98E00E94E3367090F20881E025
:1031F0008093F208F20157FC3196F595E795E80DBA
:10320000F91DAF014F505109B601D7FE02C06F5FE3
:103210007F4F759567956C0F7D1F24E030E0C501E9
:103220000E9425227092F208DF91CF911F910F9199
:10323000FF90EF90DF90CF90BF90AF909F908F90D6
:103240007F906F905F904F9008950F931F93CF934F
:10325000DF9300D000D0CDB7DEB78C012091BC0742
:103260003091BD072F5F3F4F3093BD072093BC07C0
:103270002F313105BCF0209174083091750845E379
:1032800050E060E778E0CE0101960E94E132BE0195
:103290006F5F7F4F80E798E00E943032CE01019649
:1032A0000E94AF32F801448155816081718180E7CD
:1032B00098E04533510588F40E943631F8010481C5
:1032C0001581053311055CF46DEF72E080E798E03D
:1032D0000E9422320F5F1F4FF4CF0E94363180913F
:1032E000AA07882319F11092D9081092D8081092D1
:1032F000DB081092DA088FEF9FEF9093E708809336
:10330000E6081092E9081092E80881E08093F1083D
:103310008093F0084091740850917508609170088E
:103320007091710880ED98E00E94212F26960FB6CB
:10333000F894DEBF0FBECDBFDF91CF911F910F91EB
:103340000895CF92DF92EF92FF920F931F93CF9346
:10335000DF93CDB7DEB72C970FB6F894DEBF0FBE64
:10336000CDBF6B017C018A0167EE74E0CE0101964E
:103370000E94CD32B701A601CE0101960E94933181
:103380006CE075E0CE0101960E94223220E030E030
:1033900040E151E4C701B6010E94054E20E030E053
:1033A00040EA50E40E94754F20E030E040E052E4F3
:1033B0000E94114FAB01BC01CE0101960E94633106
:1033C00061E175E0CE0101960E942232BE016F5F7D
:1033D0007F4FCE0107960E94B432CE01079635DFAB
:1033E000CE0107960E94AF3265EA77E0CE010196E2
:1033F0000E949A3264E175E0CE0101960E94223269
:10340000B801CE0101960E94F33168E874E0CE0164
:1034100001960E942232BE016F5F7F4FCE01079658
:103420000E94B432CE01079610DFCE0107960E94AB
:10343000AF32CE0101960E94AF322C960FB6F894AF
:10344000DEBF0FBECDBFDF91CF911F910F91FF90D7
:10345000EF90DF90CF900895CF92DF92EF92FF929E
:103460000F931F93CF93DF93CDB7DEB72C970FB693
:10347000F894DEBF0FBECDBF6B017C018A0166E30D
:1034800075E0CE0101960E94CD32B701A601CE01B2
:1034900001960E9493316CE075E0CE0101960E9486
:1034A000223220E030E040E151E4C701B6010E9441
:1034B000054E20E030E040EA50E40E94754F20E0E5
:1034C00030E040E052E40E94114FAB01BC01CE015C
:1034D00001960E94633161E175E0CE0101960E9480
:1034E0002232BE016F5F7F4FCE0107960E94B43239
:1034F000CE010796AADECE0107960E94AF3265EA9A
:1035000077E0CE0101960E949A326BE575E0CE011C
:1035100001960E942232B801CE0101960E94F33139
:1035200068E874E0CE0101960E942232BE016F5F0E
:103530007F4FCE0107960E94B432CE01079685DEFA
:10354000CE0107960E94AF32CE0101960E94AF32A3
:103550002C960FB6F894DEBF0FBECDBFDF91CF9192
:103560001F910F91FF90EF90DF90CF900895CF9231
:10357000DF92EF92FF920F931F93CF93DF93CDB71C
:10358000DEB72C970FB6F894DEBF0FBECDBF6B0130
:103590007C018A016DE775E0CE0101960E94CD3273
:1035A000B701A601CE0101960E9493316CE075E04F
:1035B000CE0101960E94223220E030E040E151E449
:1035C000C701B6010E94054E20E030E040EA50E419
:1035D0000E94754F20E030E040E052E40E94114F1D
:1035E000AB01BC01CE0101960E94633161E175E03F
:1035F000CE0101960E942232BE016F5F7F4FCE0145
:1036000007960E94B432CE0107961FDECE010796C0
:103610000E94AF3265EA77E0CE0101960E949A32AD
:1036200062EA75E0CE0101960E942232B801CE0115
:1036300001960E94F33168E874E0CE0101960E9481
:103640002232BE016F5F7F4FCE0107960E94B432D7
:10365000CE010796FADDCE0107960E94AF32CE0169
:1036600001960E94AF322C960FB6F894DEBF0FBEC3
:10367000CDBFDF91CF911F910F91FF90EF90DF9021
:10368000CF900895CF92DF92EF92FF920F931F9306
:10369000CF93DF93CDB7DEB72C970FB6F894DEBF8C
:1036A0000FBECDBF6B017C018A0164EC75E0CE01D9
:1036B00001960E94CD32B701A601CE0101960E946B
:1036C00093316CE075E0CE0101960E94223220E039
:1036D00030E040E151E4C701B6010E94054E20E010
:1036E00030E040EA50E40E94754F20E030E040E0D6
:1036F00052E40E94114FAB01BC01CE0101960E9421
:10370000633161E175E0CE0101960E942232BE0173
:103710006F5F7F4FCE0107960E94B432CE010796AD
:1037200094DDCE0107960E94AF3265EA77E0CE01C4
:1037300001960E949A3269EE75E0CE0101960E94D0
:103740002232B801CE0101960E94F33168E874E09C
:10375000CE0101960E942232BE016F5F7F4FCE01E3
:1037600007960E94B432CE0107966FDDCE01079610
:103770000E94AF32CE0101960E94AF322C960FB656
:10378000F894DEBF0FBECDBFDF91CF911F910F9197
:10379000FF90EF90DF90CF900895EF92FF920F93FC
:1037A0001F93CF93DF93CDB7DEB72C970FB6F89466
:1037B000DEBF0FBECDBF8091AA07882309F46CC07D
:1037C0006BE076E0CE0101960E94CD3224E1E22E3C
:1037D000F12C00E010E080E00E941C3D080F191F52
:1037E0006AE070E080E090E00E94743E21E0E21A1E
:1037F000F10889F781E00E941C3D8F3893401CF04E
:103800006EE176E021C0C80164E170E00E941D50C5
:10381000CB01770FAA0BBB0B9C01AD012C5332409F
:1038200041095109A4E6B0E00E94D54E2FE131E0F4
:1038300040E050E00E94B94EBA01A901CE010196C4
:103840000E94C33168E874E0CE0101960E942232E2
:1038500060E376E0CE0101960E942232C80164E165
:1038600070E00E941D50CE0101960E94F33169E97B
:1038700072E0CE0101960E942232BE016F5F7F4F3F
:10388000CE0107960E94B432CE010796DEDCCE014F
:1038900007960E94AF3260C064E176E0CE010196E7
:1038A0000E94CD3294E1E92EF12C00E010E080E09E
:1038B0000E941C3D080F191F6AE070E080E090E054
:1038C0000E94743E81E0E81AF10889F781E00E94C5
:1038D0001C3D8F3893401CF068E376E021C0C8019E
:1038E00064E170E00E941D50CB01770FAA0BBB0B67
:1038F0009C01AD012C53324041095109A4E6B0E0CE
:103900000E94D54E2FE131E040E050E00E94B94ED8
:10391000BA01A901CE0101960E94C33168E874E0A2
:10392000CE0101960E942232EE24EA94FE2C04E19C
:1039300010E020EA30E040E050E060EA70E080ED26
:1039400098E00E94E33622E030E042E050E062EA94
:1039500070E089819A8179D5CE0101960E94AF32BB
:103960002C960FB6F894DEBF0FBECDBFDF91CF917E
:103970001F910F91FF90EF90089565EA77E08CE733
:1039800098E00E949A3265EA77E080E798E00E942A
:103990009A321092BD071092BC0780E090E095C665
:1039A0008F929F92AF92BF92CF92DF92EF92FF924F
:1039B0000F931F93CF93DF93CDB7DEB72C970FB63E
:1039C000F894DEBF0FBECDBFEE24EA94FE2C05E4D2
:1039D00016E02CED30E040E451E064E170E080E07E
:1039E00090E0D8DB11E010930202A9D74B015C01F3
:1039F00080E011D781E00FD76B017C016CE576E0A8
:103A0000CE0107960E94CD32B501A401CE010796E2
:103A10000E94933160E776E0CE0107960E94223241
:103A2000B701A601CE0107960E94933161E175E0CE
:103A3000CE0107960E942232BE01695F7F4FCE0100
:103A400001960E94B432CE010196FFDBCE010196B1
:103A50000E94AF328091A9078823C9F181EB98E0D9
:103A60000E94BD2E6B017C0181EB98E045D69C0144
:103A7000A4E6B0E00E94014F2FEF33E040E050E0B9
:103A80000E94B94E49015A0121E7821627E19206A8
:103A9000A104B104D4F020E030E040E85FE3C701C6
:103AA000B6010E94A04D87FF10C01092A9076BE2DB
:103AB00073E0CE0101960E94CD32CE010196C5DBA6
:103AC000CE0101960E94AF3230C0A4012BC066E344
:103AD00081EB98E03DD6882341F14FDF1093A90791
:103AE00061E876E0CE0101960E94CD32CE010196CA
:103AF000ACDBCE0101960E94AF3281EB98E00E94D0
:103B0000BD2E6B017C0181EB98E0F6D59C01A4E60B
:103B1000B0E00E94014F2FEF33E040E050E00E9400
:103B2000B94EA901C701B601ADDD8091A807882370
:103B3000B9F188EA98E00E94BD2E6B017C0188EA09
:103B400098E0DAD59C01A4E6B0E00E94014F2FEF87
:103B500033E040E050E00E94B94E49015A0121375C
:103B6000374141055105D4F020E030E040E85FE303
:103B7000C701B6010E94A04D87FF10C01092A80790
:103B800069E773E0CE0101960E94CD32CE01019625
:103B90005CDBCE0101960E94AF3231C0A4012CC083
:103BA00067E388EA98E0D4D5882349F1E6DE81E02E
:103BB0008093A80763EA76E0CE0101960E94CD3299
:103BC000CE01019642DBCE0101960E94AF3288EA17
:103BD00098E00E94BD2E6B017C0188EA98E08CD5AC
:103BE0009C01A4E6B0E00E94014F2FEF33E040E0DB
:103BF00050E00E94B94EA901C701B601B8DC80911E
:103C0000A7078823C9F18FE998E00E94BD2E6B01B8
:103C10007C018FE998E070D59C01A4E6B0E00E9499
:103C2000014F2FEF33E040E050E00E94B94E4901D0
:103C30005A0121E7821627E19206A104B104D4F0CB
:103C400020E030E040E85FE3C701B6010E94A04DEC
:103C500087FF10C01092A70767EC73E0CE010196B2
:103C60000E94CD32CE010196F0DACE0101960E947B
:103C7000AF3231C0A4012CC068E38FE998E068D569
:103C8000882349F17ADE81E08093A70765EC76E02E
:103C9000CE0101960E94CD32CE010196D6DACE0138
:103CA00001960E94AF328FE998E00E94BD2E6B0111
:103CB0007C018FE998E020D59C01A4E6B0E00E9449
:103CC000014F2FEF33E040E050E00E94B94EA901D0
:103CD000C701B601C1DB8091A6078823B9F186E947
:103CE00098E00E94BD2E6B017C0186E998E004D526
:103CF0009C01A4E6B0E00E94014F2FEF33E040E0CA
:103D000050E00E94B94E49015A012137374141051F
:103D10005105D4F020E030E040E85FE3C701B60190
:103D20000E94A04D87FF10C01092A60765E174E0C5
:103D3000CE0101960E94CD32CE01019686DACE01E7
:103D400001960E94AF3231C0A4012CC069E386E91C
:103D500098E0FED4882349F110DE81E08093A60725
:103D600067EE76E0CE0101960E94CD32CE0101963B
:103D70006CDACE0101960E94AF3286E998E00E948B
:103D8000BD2E6B017C0186E998E0B6D49C01A4E6C7
:103D9000B0E00E94014F2FEF33E040E050E00E947E
:103DA000B94EA901C701B601CCDACE0107960E942F
:103DB000AF328091A907882371F081EB98E09CD401
:103DC0009C01A4E6B0E00E94014F6D3C7B4C810554
:103DD00091050CF48FC08091A807882371F088EAC0
:103DE00098E08AD49C01A4E6B0E00E94014F6D3CAB
:103DF0007B4C810591050CF4D5C08091A7078823E1
:103E000071F08FE998E078D49C01A4E6B0E00E94BC
:103E1000014F6D3C7B4C810591050CF41BC18091D9
:103E2000A607882309F46EC186E998E065D49C0151
:103E3000A4E6B0E00E94014F6D3C7B4C81059105EA
:103E40000CF060C186E998E057D49C01A4E6B0E08C
:103E50000E94014F2FEF33E040E050E00E94B94E46
:103E600002E310E0021B130B6EE777E0CE01019630
:103E70000E94CD32B801012E000C880B990B0E94D4
:103E8000A64D20E030E040E251E40E94754FAB01C6
:103E9000BC01CE0101960E9463316EE277E0CE0153
:103EA00001960E942232BE016F5F7F4FCE010796BE
:103EB0000E94B432CE010796C8D9CE0107960E945F
:103EC000AF3260E085E00E94B13C84E6809FB001A3
:103ED000819F700D1124072E000C880B990B0E94F6
:103EE000743E61E085E00E94B13CCE0101960E94E3
:103EF000AF3208C181EB98E0FFD39C01A4E6B0E0AB
:103F00000E94014F2FEF33E040E050E00E94B94E95
:103F100002E310E0021B130B69E077E0CE0101968B
:103F20000E94CD32B801012E000C880B990B0E9423
:103F3000A64D20E030E040E251E40E94754FAB0115
:103F4000BC01CE0101960E9463316EE277E0CE01A2
:103F500001960E942232BE016F5F7F4FCE0107960D
:103F60000E94B432CE01079670D9CE0107960E9406
:103F7000AF3260E082E00E94B13C84E6809FB001F5
:103F8000819F700D1124072E000C880B990B0E9445
:103F9000743E61E082E00E94B13CCE0101960E9435
:103FA000AF3219CF88EA98E0A7D39C01A4E6B0E02D
:103FB0000E94014F2FEF33E040E050E00E94B94EE5
:103FC00002E310E0021B130B64E377E0CE010196DD
:103FD0000E94CD32B801012E000C880B990B0E9473
:103FE000A64D20E030E040E251E40E94754FAB0165
:103FF000BC01CE0101960E9463316EE277E0CE01F2
:1040000001960E942232BE016F5F7F4FCE0107965C
:104010000E94B432CE01079618D9CE0107960E94AD
:10402000AF3260E083E00E94B13C84E6809FB00143
:10403000819F700D1124072E000C880B990B0E9494
:10404000743E61E083E00E94B13CCE0101960E9483
:10405000AF32D3CE8FE998E04FD39C01A4E6B0E015
:104060000E94014F2FEF33E040E050E00E94B94E34
:1040700002E310E0021B130B69E577E0CE01019625
:104080000E94CD32B801012E000C880B990B0E94C2
:10409000A64D20E030E040E251E40E94754FAB01B4
:1040A000BC01CE0101960E9463316EE277E0CE0141
:1040B00001960E942232BE016F5F7F4FCE010796AC
:1040C0000E94B432CE010796C0D8CE0107960E9456
:1040D000AF3260E084E00E94B13C84E6809FB00192
:1040E000819F700D1124072E000C880B990B0E94E4
:1040F000743E61E084E00E94B13CCE0101960E94D2
:10410000AF328DCE2C960FB6F894DEBF0FBECDBF6A
:10411000DF91CF911F910F91FF90EF90DF90CF90A3
:10412000BF90AF909F908F9008951F920F920FB6FF
:104130000F9211248F930FB6F894A8958091600088
:10414000886180936000109260000FBE8F910F9085
:104150000FBE0F901F901895CF92DF92EF92FF92B3
:10416000CF93DF93B091FC08882311F0AB2F01C0EF
:10417000A0E08091FD0890E0880F991F8A5B954D23
:10418000C0900209D0900309E0900409F09005095D
:1041900020E030E0FC01C591D491E881EB23A90136
:1041A00060E070E0EA130CC02F5F3F4F4C155D05D7
:1041B0006E057F0578F33FEF2FEF8FEF9FEF03C082
:1041C000322F252FCB01632F722FDF91CF91FF90DC
:1041D000EF90DF90CF9008959CB52091D6082CBD2C
:1041E0008EBD00000DB407FEFDCF9CBD0895CF929B
:1041F000DF92EF92FF920F931F93CF93DF93CDB790
:10420000DEB7C054D1400FB6F894DEBF0FBECDBFAD
:104210000E94AC3E0091FE081091FF082091000919
:10422000309101096B017C01C01AD10AE20AF30A3C
:1042300040EDC41647E0D406E104F10418F480917F
:104240000609C6C06093FE087093FF0880930009BA
:10425000909301091092F9081092F8081092F7084B
:104260001092F6081092F50862E08091FA080E9418
:10427000E03C61E070E080E090E00E94743E61E02C
:104280008091FA080E94E03C60E08091FA080E9468
:10429000B13C8091FB088551823028F48BE291E19A
:1042A0000197F1F706C064E170E080E090E00E94C1
:1042B000743E62E08091FA080E94E03C8091070918
:1042C00090E08230910538F0880F991F880F991F70
:1042D00005970197F1F7F89480E03EDF6F3F7F4F3D
:1042E0008F4F9F4F21F41092060978943EC081E0D1
:1042F00033DF6F3F7F4F8F4F9F4FA9F38E010F5FCB
:104300001F4F6E012FEBC21A2EEFD20A780180E008
:1043100023DFF701608371838283938381E01CDF55
:10432000F7016483758386839783F8E0EF0EF11CB1
:10433000EC14FD0461F7789420E030E0F80140814E
:10434000518162817381C480D580E680F7804F3FC0
:10435000FFEF5F076F077F0731F08FEFC816D806B2
:10436000E806F80621F41092060980E031C0F90150
:1043700083E0F595E7958A95E1F7EB50F74F80815B
:10438000880F4C155D056E057F0508F481608083FC
:104390002F5F3F4F085F1F4F2832310579F620917C
:1043A000F90830E04091F5088091F60890E0840F1C
:1043B000911D4091F708840F911D4091F808840FDA
:1043C000911D99272817390771F681E08093060916
:1043D000C05CDE4F0FB6F894DEBF0FBECDBFDF91DD
:1043E000CF911F910F91FF90EF90DF90CF900895A4
:1043F0000F931F93CF93DF93EA019C01240F351F86
:10440000215031098B01AB01BC0180ED98E00E9485
:10441000583620E0CE01009771F02EBD02D001D0B9
:1044200001C0089500002EBD0096009601D001C085
:104430000895019791F7EBE0F1E08081816080833E
:10444000DF91CF911F910F9108954F925F926F92DC
:104450007F928F929F92AF92BF92CF92DF92EF9214
:10446000FF920F931F93CF93DF931F92CDB7DEB7C9
:10447000A82F2B016A0179014091F208411107C070
:104480002091E0083091E108232B09F4A4C09701A2
:10449000225031092730310538F585E08E9DF00135
:1044A0008F9DF00D1124EE59F54DA590B49080E24A
:1044B000A81AB1082A2F392F60E070E0F901819124
:1044C0009F01882349F0F501E80FF11D87FDFA955A
:1044D000E4916E0F711DF2CF8091F108869F9001DB
:1044E000879F300D112402C020E030E085E08E9DD2
:1044F000F0018F9DF00D1124EC59F54DE491A09041
:10450000F108EA9D5001112450E0FA013197E8309A
:10451000F105E0F58827E457FF4F8F4F0C9430509A
:10452000A90156954795441A550A26C0421A530ABE
:104530002AC0A50156954795C41AD50A27C0A901D6
:1045400056954795441A550AA50156954795C41A9C
:10455000D50A12C0421A530AA50156954795C41AA6
:10456000D50A11C0CA18DB0811C0A9015695479594
:10457000441A550ACA18DB08F2E0F98309C0421A46
:10458000530ACA18DB0883E0898302C0E1E0E983AB
:1045900057FE02C0412C512C4091E2085091E30893
:1045A000B201620F731F4617570718F42A01421A07
:1045B000530AD7FE02C0C12CD12C2091E4083091BF
:1045C000E508A6014A0D5B1D2417350740F4690173
:1045D000CA18DB0804C0A12CB12CF1E0F9836A2EC3
:1045E000792E812C912CF30161913F01662379F0A2
:1045F000A201480D591D062E000C770B870196016C
:1046000080ED98E00E941B37880E991EECCF209118
:10461000E0083091E108821693060CF043C0E09068
:10462000E808F090E9088091E6089091E7088E1577
:104630009F05C1F1B201680D791DF981F23029F0B1
:10464000F33001F12819390927C02819390935959E
:1046500027958501A60180ED98E00E94E336209120
:10466000E0083091E1082819390935952795E0903F
:10467000E808F090E908C901421653060CF4C2019B
:10468000B20108C0CB01261737070CF4C9019C0101
:1046900028193909681B790B8501A60180ED98E07E
:1046A0000E94E336C4010F90DF91CF911F910F91CB
:1046B000FF90EF90DF90CF90BF90AF909F908F9042
:1046C0007F906F905F904F900895EF92FF920F93BD
:1046D0001F93E0EDF8E004891589228933897C0174
:1046E00040E050E060E070E0CF010E94E3361F91AF
:1046F0000F91FF90EF900895EF92FF920F931F9309
:10470000CF93DF931F921F92CDB7DEB728EEE22E34
:1047100023E0F22E02E09E012F5F3F4F40E16FE069
:104720000E94692D098110E0102F00278A81082B33
:1047300061E070E080E090E00E94743EC8010F905C
:104740000F90DF91CF911F910F91FF90EF900895FF
:10475000CF92DF92EF92FF920F931F93CF93DF934D
:104760001F921F92CDB7DEB76C01FC0164831FEF6F
:1047700017831092C4071092C3071092C2071092B9
:10478000C1071092C00781E08093BF071092BE0757
:1047900061E084E10E94B13C61E085E10E94B13CAE
:1047A0008091B9008E7F8093B9008091B9008D7F90
:1047B0008093B90088E48093B80085E48093BC00BE
:1047C0001A8301E09E012E5F3F4F4FE760E0C60174
:1047D0000E94123564EF71E080E090E00E94743E28
:1047E0008DE7E82EF12C9E012F5F3F4F41E060E006
:1047F000C6010E94692D998181E0953509F080E01C
:104800000F900F90DF91CF911F910F91FF90EF903C
:10481000DF90CF900895CF92DF92EF92FF92CF93E7
:10482000DF93C82FE4DC882309F47EC08091FB0865
:104830008C3009F449C018F48B30D1F075C0855123
:10484000823008F071C0D091F7086D2F6F7770E05B
:10485000762F66278091F808682B80E090E00E9410
:10486000A44D2DEC3CEC4CEC5DE30E94054E4BC09E
:104870006091F70870E080E090E00E94A44D6B0129
:104880007C01D091F808D7FF0AC09B01AC0160E021
:1048900070E080E89FEB0E94104F6B017C018D2F30
:1048A0008F70682F70E080E090E00E94A64D2DECA4
:1048B0003CEC4CEC5DE30E94054E9B01AC01C70152
:1048C000B6010E94114F21C0D091F7086D2F70E002
:1048D00080E090E00E94A44D6B017C018091F8087B
:1048E0008F70682F70E080E090E00E94A64D2DEC64
:1048F0003CEC4CEC5DE30E94054E9B01AC01C70112
:10490000B6010E94114FD7FD9058CC2389F026E6BE
:1049100036E646EE5FE30E94054E20E030E040E0E0
:1049200052E40E94114F04C060E070E080EC9FE709
:10493000DF91CF91FF90EF90DF90CF900895CF92CD
:10494000DF92EF92FF9253DC8823D1F18091FB0834
:104950008B30B0F18D30B0F08551823088F56091A8
:10496000F50870E0762F66278091F608682B80E0C6
:1049700090E00E94A44D2DEC3CEC4CEC5DE30E94D9
:10498000054E22C06091F50870E080E090E00E9442
:10499000A64D6B017C018091F608682F70E080E0E5
:1049A00090E00E94A64D2DEC3CEC4CEC5DE30E94A7
:1049B000054E9B01AC01C701B6010E94114F04C016
:1049C00060E070E080EC9FE7FF90EF90DF90CF9089
:1049D0000895CF93DF93CBE0D1E0988192609883E4
:1049E00098819E7F9883F8DB888181608883DF913E
:1049F000CF910895CF93DF939DB59093D708CBE0E7
:104A0000D1E098819D7F988398819E7F9883E4DB95
:104A1000888181608883DF91CF910895AF92BF92A2
:104A2000CF92DF92EF92FF920F931F93CF93DF937A
:104A3000EDE0F2E0A080B180C280D380C681D78152
:104A400024813581E12CF12C04E110E0A601B501AF
:104A500080ED98E00E94E336B5016C0F7D1F80EE7B
:104A6000E82E87E0F82E24E130E0A60180ED98E002
:104A70000E94E336DF91CF911F910F91FF90EF904D
:104A8000DF90CF90BF90AF9008952F923F924F92BA
:104A90005F926F927F928F929F92AF92BF92CF92CE
:104AA000DF92EF92FF920F931F93CF93DF93CDB7D7
:104AB000DEB72E970FB6F894DEBF0FBECDBF9E8730
:104AC0008D874B016A015901C801261737078CF4FD
:104AD000322F2B2DE616F7060CF004C157017B018F
:104AE000832E922E2D2D68018D859E854D872E87D4
:104AF0000DC0E216F306C4F43A2D2B2D5701E32E18
:104B0000F22E3C2D2D2D6C01832F922FA814B90469
:104B10005CF4382D292D4501A32EB22E3D852E851E
:104B2000DE86CD86C32ED22E8E149F04E9F52D8508
:104B30003E85C216D3066CF03D852E854D855E857B
:104B40004C155D0514F43C2D2D2DCD84DE843D8760
:104B50002E878C159D0544F02D853E852817390735
:104B600014F49E878D87C6014D855E85481B590BC1
:104B70004F5F5F4FB4012E960FB6F894DEBF0FBEA5
:104B8000CDBFDF91CF911F910F91FF90EF90DF90FC
:104B9000CF90BF90AF909F908F907F906F905F90DD
:104BA0004F903F902F9024CC96014D855E85241B1D
:104BB000350B3E832D8395012819390938872F83BA
:104BC0003C01641A750A9701281939093A83298327
:104BD0009C012C193D093C832B8397012A193B0921
:104BE0003A8729879501AE14BF0411F0215031098D
:104BF0008401412C512C212C312C201731077CF1C0
:104C0000C1016F8178850E941D50ED85FE85E60FFC
:104C1000F71FC20169817A810E941D504D855E8512
:104C2000640F751F8D819E81280E391E460C571CFE
:104C30006E177F072CF49E2F8F2FFB01692F782F83
:104C40006E1B7F0BAB014F5F5F4FB801CF012B870E
:104C50003C87CEDB0F5F1F4F3C852B85CECFC80135
:104C60008A199B092B813C81289F5001299FB00CF8
:104C7000389FB00C1124C80188199909689E400119
:104C8000699E900C789E900C1124E016F1069CF120
:104C9000C50169857A850E941D509601260F371F30
:104CA000C40169817A810E941D504D855E85640F23
:104CB000751F8B819C81A80EB91E860C971C6217EC
:104CC00073072CF4922F832F9B01692F782F621B7F
:104CD000730BAB014F5F5F4FB801C90189DB0F5FF9
:104CE0001F4FD3CF5B01832E922E2D2DCD84DE84DA
:104CF0004D872E8719CF2E960FB6F894DEBF0FBEC4
:104D0000CDBFDF91CF911F910F91FF90EF90DF907A
:104D1000CF90BF90AF909F908F907F906F905F905B
:104D20004F903F902F900895009769F0FC010190FB
:104D30000020E9F73197AF01481B590BBC0185EC06
:104D400097E00C94212F80E090E008958F929F923D
:104D5000AF92BF920F931F93CF93DF93CDB7DEB780
:104D6000A1970FB6F894DEBF0FBECDBF19A2423097
:104D700008F44AE08E010F5D1F4F842E912CA12C68
:104D8000B12CA50194010E94DF4EE62FB901CA01A2
:104D900001501109EA3014F4E05D01C0E95CD8016A
:104DA000EC93232B242B252B61F7C801BDDFA196A3
:104DB0000FB6F894DEBF0FBECDBFDF91CF911F912C
:104DC0000F91BF90AF909F908F900895CF92DF92F8
:104DD000EF92FF92CF93DF936B017C01E091C507C7
:104DE000F091C6070190F081E02D6DE285EC97E02F
:104DF0001995EC0166277727CB016C197D098E097F
:104E00009F094AE0A3DF8C0F9D1FDF91CF91FF9098
:104E1000EF90DF90CF900895CF93DF93BC01990F6F
:104E2000880B990B97FF02C0D1DF02C04AE08EDFEA
:104E3000EC0183EA97E078DF8C0F9D1FDF91CF9123
:104E40000895BC01990F880B990B97FDBFCF4AE0DD
:104E50007DCF8EBD00000DB407FEFDCF8EB5089549
:104E60008FEFF7CF0F93CF93DF9300D0CDB7DEB79F
:104E70006450643090F4E62FF0E0E158FD4F20815B
:104E800027FD0BC029835A834B8303E09E012F5FCC
:104E90003F4F42E068E00E9412350F900F900F9054
:104EA000DF91CF910F910895EF92FF920F931F938F
:104EB000CF93DF9300D0CDB7DEB76450643010F5E8
:104EC000E62FF0E0E558FD4F108117FD1BC0622F63
:104ED0009A017C01603151F0AFEFBFEF0E94014FAA
:104EE0002FEF30E040E050E00E94B94E19833A8342
:104EF0002B8303E09E012F5F3F4F41E068E0C70135
:104F00000E9412350F900F900F90DF91CF911F915B
:104F10000F91FF90EF9008950F931F93CF93DF931E
:104F2000EB010E94AC3E8B019BDF8F3F49F00E945A
:104F3000AC3E601B710B6C177D07B0F380E001C0C5
:104F400081E0DF91CF911F910F91089561E0FC0105
:104F500084810E94B13C80915109811110925109C4
:104F60000895CF93DF93EC018E81882379F08F81B0
:104F700098859C012F5F3F4F38872F838230924066
:104F800010F46EDFF4CFCE01E1DF1E82DF91CF910E
:104F90000895CF92DF92FF920F931F93CF93DF93E9
:104FA00000D01F92CDB7DEB76C01F62E29833A836D
:104FB0004B835C83D6DF8091510929813A814B81F3
:104FC0005C81811109C081E0809351099091620850
:104FD000809163089CBD8DBD60E0F60184812983CA
:104FE0003A834B835C830E94B13C6CE271E0C60162
:104FF00093DF8F2D80642DDF08E110E05C814B8111
:105000003A812981DA01C901002E04C0B695A7951D
:10501000979587950A94D2F729833A834B835C83CB
:1050200018DF0850110929813A814B815C81083FC2
:10503000FFEF1F0739F7FF2029F088E0F81204C0BE
:1050400087E803C085E901C08FEF03DF10E008DFC8
:10505000F601828787FF04C01F3F11F01F5FF7CF63
:105060000F900F900F900F90DF91CF911F910F91A4
:10507000FF90DF90CF900895EF92FF920F931F93D0
:10508000CF93DF93EC01790141155105610571055D
:1050900011F482E134C08B85833039F089E0440F0C
:1050A000551F661F771F8A95D1F79A01AB0168E1FA
:1050B000CE016FDF882311F084E021C08EEFC9DEBE
:1050C00087018EEFF81AF80181918F01C2DE0E156B
:1050D0001F05C9F78FEFBDDE8FEFBBDEC1DE8A870C
:1050E0008F71853029F081E18D83CE012FDF08C0DB
:1050F00068E572E0CE0110DF811106C085E18D8385
:10510000CE0124DF80E010C020E030E0A9016DE096
:10511000CE013FDF811103C0A3DE882311F084E1BB
:10512000EECFCE0113DF81E0DF91CF911F910F9180
:10513000FF90EF900895CF93DF93809154098823D7
:1051400089F1C0915209D0915309409115025091B3
:105150001602609117027091180229E539E0CE011C
:105160008BDF811102C080E01EC040915509509133
:10517000560960915709709158094115510561050B
:10518000710571F029E539E0CE0176DF882359F306
:105190001092550910925609109257091092580909
:1051A0001092540981E0DF91CF910895BF92CF9280
:1051B000DF92EF92FF920F931F93CF93DF936B01D8
:1051C0007C01B42E8091150290911602A0911702D5
:1051D000B09118028C159D05AE05BF0509F46FC08E
:1051E000AADF882309F472C0C0915209D0915309F3
:1051F0008E81882369F088819981AA81BB81C81634
:10520000D906EA06FB0621F48F819885892B99F14E
:10521000C882D982EA82FB828B85A70196018330FE
:1052200039F089E0220F331F441F551F8A95D1F7AB
:1052300061E1CE01AEDE882319F083E08D8333C0B7
:105240000E94AC3E8B010CDE8A878F3F49F40E949E
:10525000AC3E601B710B6D327140A8F38FE003C050
:105260008E3F29F08DE08D83CE0170DE1CC0188644
:105270001F8281E08E8309E519E0F2DDF801819358
:105280008F01FBE009351F07C1F78F8198859E5F6D
:1052900098878F832985222319F08115924038F051
:1052A000CE015FDE04C0CE0151DE80E00FC0C092AF
:1052B0001502D0921602E0921702F0921802809125
:1052C0005409482F4B294093540981E0DF91CF9135
:1052D0001F910F91FF90EF90DF90CF90BF900895B6
:1052E0004F925F926F927F928F929F92AF92BF92F6
:1052F000CF92DF92EF92FF920F931F93CF93DF93A2
:10530000EC016A017B012801390142305105610538
:10531000710510F480E072C089859A85AB85BC85E3
:105320000196A11DB11D84179507A607B70790F335
:105330008B889C88AD88BE888F89803129F4BB27F3
:10534000AF2D9E2D8D2D09C0DB01CA0147E0B6951A
:10535000A795979587954A95D1F7880E991EAA1E0D
:10536000BB1E8091150290911602A0911702B09178
:10537000180288169906AA06BB0679F48F8980312F
:1053800099F4DD24EE24FF24C601880F991FFC0147
:10539000E75AF64F5182408218C040E0C501B4017F
:1053A00005DF8111EBCFB6CFE894C7F8DD24EE24FA
:1053B000FF24C601880F991F880F991FFC01E75A27
:1053C000F64F4082518262827382809154098160DB
:1053D000809354098A89823080F08D819E81AF81CB
:1053E000B885880E991EAA1EBB1E80925509909200
:1053F0005609A0925709B092580981E0DF91CF91E8
:105400001F910F91FF90EF90DF90CF90BF90AF90E2
:105410009F908F907F906F905F904F9008958F92A4
:105420009F92AF92BF92CF92DF92EF92FF920F9333
:105430001F93CF93DF93FC0181859285A385B4856B
:105440000196A11DB11D84179507A607B70710F493
:1054500080E05BC083899489A589B689C789C031FA
:1054600029F4852E962EA72EBB2409C04A015B0184
:10547000C7E0B694A79497948794CA95D1F7E901A9
:105480006A017B018F01BC01CD01680D791D8A1D68
:105490009B1D8090150290901602A0901702B0906C
:1054A0001802681579058A059B0599F4F801878922
:1054B0008031A1F4B701A601552766277727440F4D
:1054C000551FFA01E75AF64F80819181A0E0B0E0C4
:1054D00017C040E06BDE8111E9CFBACFB701A6015A
:1054E0004F77552766277727440F551F440F551FC1
:1054F000FA01E75AF64F80819181A281B381BF7092
:1055000088839983AA83BB8381E0DF91CF911F9128
:105510000F91FF90EF90DF90CF90BF90AF909F9052
:105520008F9008953F924F925F926F927F928F92E9
:105530009F92AF92BF92CF92DF92EF92FF920F9322
:105540001F93CF93DF93CDB7DEB72C970FB6F894A8
:10555000DEBF0FBECDBF5C01DC015B968D909C90E1
:105560005C971696CD90DD90ED90FC901997C11444
:10557000D104E104F10439F0BFEFCB1ADB0AEB0AE6
:10558000FB0A312C07C0F401C080D180E280F38097
:1055900033243394F40181859285A385B4859C01DD
:1055A000AD012F5F3F4F4F4F5F4F29873A874B87A2
:1055B0005C87260137011D821E821F821886F40136
:1055C00081859285A385B4852D813E814F81588543
:1055D000281739074A075B0708F060C089859A8554
:1055E000AB85BC858C159D05AE05BF0550F482E0EA
:1055F000C82ED12CE12CF12C92E0492E512C612C9B
:10560000712C9E012F5F3F4FB701A601C40107DF38
:10561000882309F443C089819A81AB81BC81892B9D
:105620008A2B8B2B41F0260137019FEF491A590A2B
:10563000690A790A05C0C414D504E604F70491F098
:105640002D813E814F8158852F5F3F4F4F4F5F4FD8
:105650002D833E834F8358873FEFC31AD30AE30A53
:10566000F30AADCF0FEF1FEF2FEF3FE0B301A20121
:10567000C40136DE882391F0D50116964D915D91D7
:105680006D917C911997411551056105710541F0A6
:1056900093018201C40124DE811102C080E02AC08E
:1056A000D50116964D925D926D927C92199733209A
:1056B00051F0D301C2010196A11DB11DF4018083F7
:1056C0009183A283B383F5018789908DA18DB28DDB
:1056D000892B8A2B8B2B69F4D50157964D925D92BD
:1056E0006D927C925A9714968C91149780681496B8
:1056F0008C9381E02C960FB6F894DEBF0FBECDBF21
:10570000DF91CF911F910F91FF90EF90DF90CF909D
:10571000BF90AF909F908F907F906F905F904F90D1
:105720003F9008954F925F926F927F928F929F92D7
:10573000AF92BF92EF92FF920F931F93CF93DF939D
:1057400000D01F921F92CDB7DEB78C016D83DC01B4
:1057500015968C911597813009F056C014968C914E
:1057600081FF52C059C0038CF48DE02D258530E0B7
:10577000275F3F4F2A013B01B1E04B1A51086108F6
:105780007108022E04C076946794579447940A9443
:10579000D2F7D501C4010197A109B10904C0B6959A
:1057A000A795979587952A95D2F784159505A6050F
:1057B000B70508F06FC0F8014789508D618D728D73
:1057C00046835783608771872C013D017801E6E0AD
:1057D000EE0EF11CD801411451046104710409F466
:1057E00063C016964D915D916D917C9119979701CB
:1057F0005B968D919C915C9712DEB1E04B1A51083B
:10580000610871088111E6CF81E090E0F80193838F
:10581000828380E090E049C182FF0EC0F80142859A
:1058200053856485758583889488A588B6884815CE
:1058300059056A057B05F1F4D8011A964D915D91E1
:105840006D917C911D975B968D919C915C97FC016D
:1058500074807A944A015B0129E0B694A7949794E6
:1058600087942A95D1F778207A01F1E0FF227720FA
:1058700011F162C081149104A104B10409F073CF45
:105880001682178210861186F801128613861486F6
:105890001586D2CF452B462B472B09F48CCF841984
:1058A0009509A609B70990CF1A968D929D92AD924F
:1058B000BC921D97C1CFE114F10409F03DC0F8017D
:1058C00046815781608571854115510561057105D6
:1058D00049F48789908DA18DB28D0097A105B105FE
:1058E00031F520C09E012F5F3F4F99DD882309F4D9
:1058F00090CF89819A81AB81BC81F801238D348D51
:10590000F9012789203129F048EF5FEF6FEF7FE041
:1059100004C048EF5FEF60E070E084179507A607CA
:10592000B70728F0C801FEDD811106C06DCFF80170
:1059300086839783A087B187D8015B96ED91FC9110
:105940005C9716968D909D90AD90BC901997B2E0A3
:105950008B1A9108A108B108058404C0880C991C11
:10596000AA1CBB1C0A94D2F786859785A089B189A9
:10597000880E991EAA1EBB1E870C911CA11CB11C6F
:10598000E114F10401F5F8014285538564857585BC
:1059900083899489A589B689481759076A077B07BF
:1059A00090F0C9DB882309F42FCF809215029092E2
:1059B0001602A0921702B0921802809154098160D9
:1059C0008093540907C041E0C501B401EFDB88238F
:1059D00009F41ACFF701E75AF64F8D818083F80159
:1059E00082859385A485B5850196A11DB11D828709
:1059F0009387A487B5874389548965897689481731
:105A000059076A077B0738F4838B948BA58BB68B79
:105A1000848180688483D80114968C9183FD03C0AF
:105A200081E090E042C0F8019581992309F4ECCE21
:105A300087FF37C0668577858089918941E0B6DB2D
:105A4000882309F4E1CED8015296EC91B0E2EB9FA5
:105A500090011124D901A75AB64F109709F4D4CE5A
:105A6000F8018581823050F44389548965897689AB
:105A70005C964D935D936D937C935F97F801878956
:105A8000908DA18DB28DF901E75AF64F938F828FD9
:105A9000B58BA48BD80114968C9114978F7714969C
:105AA0008C9349DB8111BCCFAFCE0F900F900F903C
:105AB0000F900F90DF91CF911F910F91FF90EF907A
:105AC000BF90AF909F908F907F906F905F904F901E
:105AD00008952F923F924F925F926F927F928F9292
:105AE0009F92AF92BF92CF92DF92EF92FF920F936D
:105AF0001F93CF93DF9300D000D0CDB7DEB79E8346
:105B00008D83562E442E3C832B834701C701880F7B
:105B1000991F880F991F3C0125E0621A710810E057
:105B2000FF24F394202E312C35ECE32E101708F0CF
:105B3000CDC0AD81BE8114968C911497F0925A0B12
:105B40008093590B1092C2071092C10715968D9140
:105B50009C911697DC01ED91FC910190F081E02D74
:105B6000652D1995ED81FE8185819681DC01ED9190
:105B7000FC910190F081E02D642D1995ED81FE815D
:105B800087818F3F79F4AD81BE8115968D919C916F
:105B90001697EBD6B2E08B16910460F0C301019723
:105BA000F1F708C0ED81FE8187810E94893C892B35
:105BB000C9F3E9CFAD81BE8117968C918F3F21F457
:105BC000ED81FE81348109C0AD81BE8117968C9133
:105BD0000E94893C892BC1F3F3CF8091C0078111CA
:105BE000FCCFC101811B91098132910514F080E243
:105BF00090E0282F813208F020E2F092C007F09266
:105C0000BF07BFEFB0937B0B10929D0B4FEF420F7E
:105C100040939C0BF0929E0B40919E0B330F342BC4
:105C200030939E0B3091BE07313069F41092BE075D
:105C300030919E0B3093BB003091BC0033FDF8CF08
:105C4000E092BC0003C0E5EEE093BC003091C007D9
:105C50003130E1F330919D0B321710F420919D0B00
:105C6000ACE7BBE0EBE5FBE03E2F4BE55BE0341B34
:105C7000321718F43D913193F7CF1092C407209357
:105C8000C307A12CB12C6C01DD24812F8A0DAC142B
:105C9000BD04D4F42B813C81280F311D3A83298324
:105CA000AD81BE8115968D919C911697DC01ED9189
:105CB000FC910284F385E02D1995E981FA818083B6
:105CC000FFEFAF1ABF0AE1CF182F30CF26960FB6DD
:105CD000F894DEBF0FBECDBFDF91CF911F910F9122
:105CE000FF90EF90DF90CF90BF90AF909F908F90FC
:105CF0007F906F905F904F903F902F900895EF921C
:105D0000FF920F931F93CF93DF931F921F92CDB7F4
:105D1000DEB7633059F020F4623021F540E009C06D
:105D2000643031F06530F1F443E003C041E001C07C
:105D300042E0495F24EFE22EFF24F39402E09E014B
:105D40002F5F3F4F69E0C5DE098110E0102F00276B
:105D50008A81082B61E070E080E090E00E94743E50
:105D6000C80102C080E090E00F900F90DF91CF91CA
:105D70001F910F91FF90EF900895EF92FF920F9374
:105D8000CF93DF9300D01F92CDB7DEB728EEE22E7F
:105D900023E0F22E04E09E012F5F3F4F44E060E0DD
:105DA00098DE29816A81862F90E0A0E0B0E0DC01D6
:105DB00099278827B22B2C81822B2B81BC01CD0106
:105DC000722B0E94A64D20E030E040E857E30E948D
:105DD000054E0F900F900F900F90DF91CF910F9184
:105DE000FF90EF900895EF92FF920F93CF93DF9380
:105DF00000D01F92CDB7DEB72DE7E22EF12C04E0E4
:105E00009E012F5F3F4F42E060E063DE29816A819F
:105E1000862F90E0A0E0B0E0DC0199278827B22B24
:105E20002C81822B2B81BC01CD01722B0F900F9006
:105E30000F900F90DF91CF910F91FF90EF90089509
:105E40000895CF92DF92EF92FF920F931F93CF931B
:105E5000DF936C017A018B01C0E0D0E0CE15DF0545
:105E600089F0D8016D918D01D601ED91FC910190E1
:105E7000F081E02DC6011995892B11F47E0102C035
:105E80002196ECCFC701DF91CF911F910F91FF9029
:105E9000EF90DF90CF900895FC01538D448D252F16
:105EA00030E0842F90E0821B930B541710F0CF96B4
:105EB000089501970895FC01918D828D981761F0E6
:105EC000828DDF01A80FB11D5D968C91928D9F5F31
:105ED0009F73928F90E008958FEF9FEF0895FC01DC
:105EE000918D828D981731F0828DE80FF11D858D8F
:105EF00090E008958FEF9FEF0895FC01918D228D22
:105F0000892F90E0805C9F4F821B91098F739927A6
:105F1000089585EC97E0F1DF21E0892B09F420E07A
:105F2000822F0895FC01848DDF01A80FB11DA35AB3
:105F3000BF4F2C91848D90E001968F739927848FA9
:105F4000A689B7892C93A089B1898C9180648C93A0
:105F5000938D848D981306C00288F389E02D80818B
:105F60008F7D80830895EF92FF920F931F93CF93BD
:105F7000DF93EC0181E0888F9B8D8C8D981305C099
:105F8000E889F989808185FD23C0F62E0B8D10E00C
:105F90000F5F1F4F0F731127E02E8C8DE8120BC07F
:105FA0000FB607FCFACFE889F989808185FFF5CF24
:105FB000CE01B8DFF2CF8B8DFE01E80FF11DE35A61
:105FC000FF4FF0820B8FEA89FB898081806207C0D6
:105FD000EE89FF896083E889F98980818064808304
:105FE00081E090E0DF91CF911F910F91FF90EF90B2
:105FF0000895CF93DF93EC01888D8823C1F0EA895F
:10600000FB89808185FD05C0A889B9898C9186FDB1
:106010000EC00FB607FCF5CF808185FFF2CFA889AF
:10602000B9898C9185FFEDCFCE017CDFE8CFDF9180
:10603000CF91089580E090E0892B19F06ADF8111FB
:1060400025C080E090E0892B41F080E090E0892B32
:1060500021F00E94000081111CC080E090E0892B9B
:1060600041F080E090E0892B21F00E940000811136
:1060700013C080E090E0892BA1F080E090E0892BB4
:1060800081F00E94000081110AC008950E94000062
:10609000D8CF0E940000E1CF0E940000EACF0C940C
:1060A0000000089585ED8093BC008091BC0084FDC4
:1060B000FCCF1092C00708954091E10B262F30E0ED
:1060C000240F311D21323105DCF42091C00724302A
:1060D000C9F4FC0180E090E0861758F43091E10BA0
:1060E0002191DC01A154B44FA30FB11D2C93019653
:1060F000F3CF8091E10B680F6093E10B80E008958E
:1061000081E0089582E008950895E091C4078091A8
:10611000C307E81730F4F0E0E55AF44F808190E0CF
:1061200008958FEF9FEF08959091C4078091C30762
:10613000981750F4E92FF0E0E55AF44F208130E051
:106140009F5F9093C40702C02FEF3FEFC9010895EE
:106150008091C30790E02091C407821B91090895A4
:10616000CF92DF92EF92FF920F931F93CF93DF9323
:106170007C01262F972F8A0180915A0B882391F05A
:10618000C62FD72F6E01C40ED51ECC15DD0569F0C4
:106190006991D701ED91FC910190F081E02DC7014B
:1061A0001995F3CF642F822F87DFC801DF91CF913C
:1061B0001F910F91FF90EF90DF90CF900895CF93B4
:1061C000DF931F92CDB7DEB7698320915A0B22234C
:1061D000D1F02091C107203240F021E030E0FC01F5
:1061E0003383228380E090E014C08091C207E82FBF
:1061F000F0E0E156F44F998190838F5F8093C2075E
:106200008093C10704C061E0CE01019655DF81E0B3
:1062100090E00F90DF91CF9108950E9463520F9309
:106220001F93CF93DF93EC0188819981009729F028
:106230002A813B812617370788F48B016F5F7F4FD8
:106240000E947F51009761F0998388831B830A83A2
:106250002C813D81232B11F4FC01108281E001C0CF
:1062600080E0DF91CF911F910F910895EF92FF92FF
:106270000F931F93CF93DF93FC0124813581611528
:10628000710511F480E018C041155105A1F07B01A2
:10629000EC018A01020F131FB801C1DF882391F3BB
:1062A000288139818C819D81B701820F931F0E94C3
:1062B00070521D830C8381E0DF91CF911F910F916C
:1062C000FF90EF900895EF92FF920F931F93CF935B
:1062D000DF93CDB7DEB764970FB6F894DEBF0FBE7D
:1062E000CDBF7C01CB01BA018E010F5F1F4F22E0B1
:1062F00044E00E94BA4ABC01FC0101900020E9F789
:106300003197AF01481B590BC701B0DF64960FB638
:10631000F894DEBF0FBECDBFDF91CF911F910F91DB
:10632000FF90EF900895EF92FF920F931F93CF93FA
:10633000DF93CDB7DEB764970FB6F894DEBF0FBE1C
:10634000CDBF7C01CB01BA018E010F5F1F4F22E050
:1063500044E00E94BA4ABC01FC0101900020E9F728
:106360003197AF01481B590BC70180DF64960FB608
:10637000F894DEBF0FBECDBFDF91CF911F910F917B
:10638000FF90EF900895EF92FF920F931F93CF939A
:10639000DF93CDB7DEB72E970FB6F894DEBF0FBEF2
:1063A000CDBF7C01CB01BA012AE08E010F5F1F4FE8
:1063B000A8010E94E34AF80101900020E9F7319713
:1063C000AF01401B510BB801C70150DF2E960FB62D
:1063D000F894DEBF0FBECDBFDF91CF911F910F911B
:1063E000FF90EF900895EF92FF920F931F93CF933A
:1063F000DF93CDB7DEB728970FB6F894DEBF0FBE98
:10640000CDBF7C01CB014AE08E010F5F1F4FB80169
:106410000E94D94AF80101900020E9F73197AF01B5
:10642000401B510BB801C70121DF28960FB6F89425
:10643000DEBF0FBECDBFDF91CF911F910F91FF90B7
:10644000EF9008956115710549F0FB01019000205E
:10645000E9F73197AF01461B570B08CF80E008954D
:106460000F931F93CF93DF938C01EB01FC0180818D
:1064700091810097B1F0688179816115710579F09A
:10648000428153812C813D814217530740F00E9485
:1064900070528C819D81F8019583848313C00E9482
:1064A000E75088819981F801918380838A819B815B
:1064B000938382838C819D81958384831982188242
:1064C0001B821A821D821C82DF91CF911F910F9136
:1064D0000895CF93DF93EC0188819981009711F0A3
:1064E0000E94E750198218821D821C821B821A8228
:1064F000DF91CF910895EF92FF920F931F93CF9367
:10650000DF93EC017B018A01BA0189DE811103C0AE
:10651000CE01DFDF07C01D830C83B701888199811D
:106520000E947052CE01DF91CF911F910F91FF9089
:10653000EF900895CF93DF93EC016115710551F051
:10654000FB0101900020E9F73197AF01461B570B83
:10655000D2DF01C0BEDFCE01DF91CF910895FC01F3
:10656000808191810C94E750FB01DC0111961C9213
:106570001E9213961C921E92129715961C921E92B2
:1065800014978617970741F0608171816115710535
:1065900019F044815581AFCF0895FC01118210821A
:1065A00013821282158214826115710549F0FB0174
:1065B00001900020E9F73197AF01461B570B9BCFA5
:1065C0000895BF92CF92DF92EF92FF920F931F93A5
:1065D000CF93DF937C016B018A01E9012417350712
:1065E00020F4812F8901C42FD82F65EA77E0C701F5
:1065F000D4DFD60114968D919C9115970817190731
:10660000C8F48C179D0708F4EC01D601ED91FC91BC
:106610001197EC0FFD1FB08010824D915C91BA0173
:10662000600F711FC70186DFD601ED91FC91EC0F61
:10663000FD1FB082C701DF91CF911F910F91FF9095
:10664000EF90DF90CF90BF9008951F920F920FB6FA
:106650000F9211240BB60F922F933F934F935F939A
:106660006F937F938F939F93AF93BF93EF93FF931A
:1066700085EC97E057DCFF91EF91BF91AF919F912F
:106680008F917F916F915F914F913F912F910F90DB
:106690000BBE0F900FBE0F901F9018951F920F9278
:1066A0000FB60F9211240BB60F922F938F939F93D7
:1066B000EF93FF93E091D507F091D6078081E091A9
:1066C000DB07F091DC0782FD12C090818091DE072C
:1066D0008F5F8F732091DF07821751F0E091DE0703
:1066E000F0E0EB53F84F958F8093DE0701C0808177
:1066F000FF91EF919F918F912F910F900BBE0F9073
:106700000FBE0F901F9018951F920F920FB60F9209
:1067100011240BB60F922F933F934F935F936F9378
:106720007F938F939F93AF93BF93EF93FF9380914A
:10673000B900887F803609F49CC068F5883209F476
:106740005BC090F4803109F454C038F4882309F414
:10675000F6C0883009F44DC0F5C0883109F44CC04A
:10676000803209F45DC0EEC0803409F468C048F49A
:10677000803309F455C0883309F0E4C080937B0B63
:10678000D8C0803509F44FC0883509F45DC088341D
:1067900009F0D8C0D6C0883909F4C7C0A8F4883732
:1067A00009F467C038F4883609F463C0803709F407
:1067B00060C0C8C0883809F4B8C0803909F45FC027
:1067C000803809F0BFC05BC0803B09F486C038F454
:1067D000803A09F466C0883A09F47FC0B3C0803CAF
:1067E00009F4A7C0883C09F4A4C0883B09F48AC016
:1067F000A9C080919E0B10C090919D0B80919C0B25
:10680000981770F5E0919D0B81E08E0F80939D0BA2
:10681000F0E0E458F44F80818093BB0085EC86C0A3
:1068200080937B0B8EC0E0919D0B81E08E0F809357
:106830009D0B8091BB00F0E0E458F44F8083909171
:106840009D0B80919C0B6EC0E0919D0B81E08E0FA3
:1068500080939D0B8091BB00F0E0E458F44F80835F
:106860008091BF0781116DC081E08093BE0784EAEB
:1068700061C083E08093C0071092050CCFCF809158
:10688000050C803208F051C0E091050C81E08E0FBC
:106890008093050C8091BB00F0E0EB51F44F8083B6
:1068A000BDCF85EC8093BC001092C0078091050C91
:1068B000803230F4E091050CF0E0EB51F44F10829F
:1068C0006091050C70E0E091E30BF091E40B85EE34
:1068D0009BE019951092050C35C084E08093C007A9
:1068E0001092E20B1092E10BE091DF0BF091E00BC4
:1068F00019958091E10B811105C081E08093E10B36
:106900001092BF0BE091E20B81E08E0F8093E20BBF
:10691000F0E0E154F44F80818093BB009091E20B52
:106920008091E10B981708F479CF85E88093BC003B
:1069300009C085EC8093BC001092C00703C0109280
:106940007B0BB0DBFF91EF91BF91AF919F918F9146
:106950007F916F915F914F913F912F910F900BBE5F
:106960000F900FBE0F901F9018952091C107909126
:10697000590B213208F04AC08091C0078111FCCF29
:1069800032E03093C00731E03093BF073FEF3093E0
:106990007B0B10929D0B20939C0BAFE9BBE04CE767
:1069A0005BE0FA013E2F341B321718F43D9131930E
:1069B000F9CF10929E0B20919E0B990F922B9093E2
:1069C0009E0B9091BE07913061F41092BE0790919A
:1069D0009E0B9093BB009091BC0093FDF8CF95EC7B
:1069E00001C095EE9093BC009091C0079230E1F306
:1069F00090917B0B9F3F79F080917B0B803241F02F
:106A000080917B0B803331F084E005C081E003C0CE
:106A100082E001C083E01092C2071092C107109279
:106A20005A0B0895CF92DF92EF92FF920F93CF937C
:106A3000DF931F92CDB7DEB76C017901DC011496AC
:106A40008C91149791E090935A0B8093590B10926C
:106A5000C2071092C10715968D919C911697DC0183
:106A6000ED91FC910190F081E02D49831995F6019B
:106A700085819681DC01ED91FC910190F081E02D02
:106A80004981642F1995F60185819681DC01ED918C
:106A9000FC91402F50E00280F381E02DB701199561
:106AA000F60187818F3F71F4D60115968D919C91E7
:106AB00016970F90DF91CF910F91FF90EF90DF909D
:106AC000CF9053CFF601878124D7892BD9F3ECCF10
:106AD000CF92DF92EF92FF920F93CF93DF93CDB7D8
:106AE000DEB7A0970FB6F894DEBF0FBECDBF6C0126
:106AF000862FFB010E2F081B9191E02EF12C99237C
:106B000041F0A1E0B0E0AC0FBD1FAE0DBF1D9C93E6
:106B1000F1CF9E012F5F3F4F45E062E0C60182DF6B
:106B2000C701A0960FB6F894DEBF0FBECDBFDF91B0
:106B3000CF910F91FF90EF90DF90CF9008950F933A
:106B4000CF93DF931F92CDB7DEB7698301E09E013B
:106B50002F5F3F4F45E062E065DF61E070E080E07D
:106B600090E00E94743E81E090E00F90DF91CF9121
:106B70000F910895FC01828993896817790708F0BD
:106B800096C0848995894817590708F090C080916C
:106B90000B018E7F80930B01868D978D861797074B
:106BA00009F42BC080910B018D7F80930B018AE249
:106BB0008EBD0000009601D001C00895778F668FCA
:106BC00080910B01826080930B017EBD02D001D0C9
:106BD00001C0089500006EBD02D001D001C008952B
:106BE00000007EBD02D001D001C0089500006EBD3E
:106BF0000000009601D001C00895848D958D841702
:106C0000950709F42CC080910B018D7F80930B01B7
:106C10008BE28EBD0000009601D001C00895558F13
:106C2000448F80910B01826080930B015EBD02D086
:106C300001D001C0089500004EBD02D001D001C0B6
:106C4000089500005EBD02D001D001C0089500008B
:106C50004EBD00000096009601D001C008958091BD
:106C60000B018D7F80930B018CE28EBD0096009608
:106C7000009601D001C0089580910B01826080933D
:106C80000B013EBD00960096009601D001C008950C
:106C9000758764872EBD0000009601D001C008955D
:106CA0005787468780910B01816080930B0108957F
:106CB0000F931F93FC0180910B018D7F80930B013B
:106CC00080910B018E7F80930B018AE28EBD00962E
:106CD0000096009601D001C0089580910B0182605A
:106CE00080930B017EBD0000009601D001C0089585
:106CF0008FEF9FEF978F868F6EBD0000009601D0BB
:106D000001C00895848595852817390781F03EBD17
:106D10000000009601D001C0089500003587248747
:106D20002EBD00000096009601D001C0089580910C
:106D30000B018D7F80930B018BE28EBD0096009638
:106D4000009601D001C0089580910B01826080936C
:106D50000B015EBD0000009601D001C008958FEFC9
:106D60009FEF958F848F4EBD0000009601D001C02B
:106D70000895868597850817190781F01EBD0000C4
:106D8000009601D001C008950000178706870EBD48
:106D900000000096009601D001C0089580910B017B
:106DA0008D7F80930B018CE28EBD000000960096D3
:106DB00001D001C0089580910B01826080930B0186
:106DC0001F910F910895CF92DF92EF92FF920F9350
:106DD0001F93CF93DF936901E8018A010C0F1D1FF8
:106DE00001501109FB01E20FF31F9F0121503109EE
:106DF0005FDF219790F0C601009771F0FEBC02D0D2
:106E000001D001C008950000EEBC0096009601D0AC
:106E100001C00895019791F7ECCF80910B0181603B
:106E200080930B01DF91CF911F910F91FF90EF9015
:106E3000DF90CF9008952F923F924F925F926F9282
:106E40007F928F929F92AF92BF92CF92DF92EF92FA
:106E5000FF920F931F93CF93DF93CDB7DEB7669763
:106E60000FB6F894DEBF0FBECDBF1C0158874F830D
:106E70002901FC01008CF18DE02DFC87EB87FC01E2
:106E8000C688D7880130110509F0FDC0F1A1FD8742
:106E9000FC0182899389481759070CF0EDC0848959
:106EA0009589281739070CF0E7C0FD85AF2EB12C66
:106EB000CA0106E0F09F800D911D112418161906D5
:106EC0000CF0DAC0C501E3E0880F991FEA95E1F7FD
:106ED000840D951D181619060CF0CEC031E0398BC3
:106EE0004B855C854C155D0509F4198A7B01FF24EF
:106EF0005D85513009F05DC06989662309F459C088
:106F00008201085F1F4F2F8138852B5F3F4FA20101
:106F10006F817885C101CCDE85E08E9DA0018F9DBB
:106F2000500D11249E012F5F3F4FD90180E090E06A
:106F3000FC01E40FF51FED5CF44DE491ED93019637
:106F400085309105A9F71E826D2D5C8598E081E062
:106F500075E0720FF9014191482351F00DB407FE1D
:106F6000FDCF6EBD00000DB407FEFDCFCEBC0AC044
:106F70000DB407FEFDCF5EBD00000DB407FEFDCFD2
:106F80000B850EBD7E13E7CF880F0DB407FEFDCF36
:106F90005EBD0DB407FEFDCF4B854EBD9150D1F6C1
:106FA0000DB407FEFDCF80910B01816080930B0132
:106FB00063C085E08E9DB0018F9D700D11247E8B86
:106FC0006D8B8F819885988B8F87812C912C95E084
:106FD0008916910449F0ED89FE89E80DF91DED5CF3
:106FE000F44D0491098701C019862D85213029F5BA
:106FF000720118E06F807884680C791C398530FF45
:1070000005C09601A701B301C101B4DD49854695CC
:10701000498711505FEFE51AF50A1111EFCF6FEFB5
:10702000861A960A8F8598898A0D9B1D988B8F8763
:1070300096E08916910459F61FC03201E8E0EB8B07
:10704000F985F0FF02C0760105C00989002349F0E7
:10705000EB84FC8485019501A3016F857889C101CA
:10706000B2DE2985269529873B8931503B8B6A0CF6
:107070007B1C3111E5CFD3CFF10181A1F6E08F9FC9
:10708000C00111242AC360527109CB01880F991FD6
:107090000230110599F4FC01EA57F64D259134911F
:1070A0003E872D87FB01EA5DF64DE4914E2F50E0BF
:1070B0005A87498740E1642E712C25C045E0409FE6
:1070C0009001419F300D1124F901E05AF54D459191
:1070D0005491FA01E80FF91F859194919E878D874D
:1070E000F901EE59F54D85919491FC01E60FF71FDA
:1070F000E4914E2F50E05A874987F901EC59F54D3C
:10710000E4916E2E712CC98ADB8A0230110509F0D8
:10711000C5C1F10121A149855A85249FC001259F40
:10712000900D11246F817885680F791F42895389EA
:10713000641775070CF0D1C289859A850696BC0143
:1071400033E0759567953A95E1F7788B6F878B8576
:107150009C85C816D90619F0213009F447C11C8A4C
:107160001B8A1A8A198A69897A896615770509F44A
:10717000ABC2F101E08CF18C868997898E159F0551
:1071800081F001A110E049855A85409F9001419FFF
:10719000300D509F300D1124A2016F817885C101FF
:1071A00012DE6B897C898D859E85680F791F7E8BA9
:1071B0006D8BAF80B8841C861B864B855C856F8584
:1071C00078894617570709F400C1EB85FC852D899E
:1071D0003E89E20FF31F9490992009F4ECC0F1016D
:1071E00021A1213009F056C097FE06C026893789B3
:1071F000A201B501C101BEDC96FE09C0F1012689DC
:107200003789A201B5016F5F7F4FC101B3DC95FEE5
:1072100009C0F10126893789A201B5016E5F7F4F50
:10722000C101A8DC94FE09C0F10126893789A201B9
:10723000B5016D5F7F4FC1019DDC93FE09C0F10177
:1072400026893789A201B5016C5F7F4FC10192DCAD
:1072500092FE09C0F10126893789A201B5016B5F51
:107260007F4FC10187DC91FE09C0F1012689378972
:10727000A201B5016A5F7F4FC1017CDC90FE9BC01B
:10728000F10126893789A201B501695F7F4FC101EC
:1072900071DC91C030E0C5014F815885841B950B8E
:1072A000829F6001839FD00C929FD00C1124C40E4A
:1072B000D51E97FE08C0F101E688F7888901A20172
:1072C000B601C10180DD96FE0CC0F10121A130E0C4
:1072D000E688F788B601620F731F8901A201C10118
:1072E00072DD95FE0EC0F10121A130E0E688F7883D
:1072F000B901660F771F6C0D7D1D8901A201C101C7
:1073000062DD94FE10C0F10181A1282F30E0E688F3
:10731000F788B601F3E08F9F600D711D112489017C
:10732000A201C10150DD93FE10C0F10181A1E688E8
:10733000F788282F30E0B601F4E08F9F600D711DB3
:1073400011248901A201C1013EDD92FE10C0F101AC
:1073500081A1282F30E0E688F788B601F5E08F9FFD
:10736000600D711D11248901A201C1012CDD91FE66
:1073700010C0F10181A1282F30E0E688F788B6011E
:10738000F6E08F9F600D711D11248901A201C101DA
:107390001ADD90FE10C0F10181A1282F30E0E688AF
:1073A000F788B601F7E08F9F600D711D11248901E8
:1073B000A201C10108DD2B853C852F5F3F4F3C8733
:1073C0002B8738E0A30EB11CF8CEF10181A1480E45
:1073D000511C29893A892F5F3F4F3A8B298B4B8962
:1073E0005C89460F571F5C8B4B8BBDCE8201060D0F
:1073F000171D015011092F85388983E0220F331F93
:107400008A95E1F78F819885280F391F215031091E
:10741000A201BC01C1014CDC1C8520E030E040E051
:1074200050E04615570509F435C0AD85BE85A20F5D
:10743000B31F80E090E06F8578898617970729F160
:10744000FC01EA0FFB1FE49168E070E0F0E80F2F09
:107450000E2359F00DB407FEFDCF0B890EBD0000C1
:107460000DB407FEFDCF098909C00DB407FEFDCF9D
:107470001EBD00000DB407FEFDCF0B850EBDF695B9
:107480006150710921F70196D6CF4F5F5F4F260FEC
:10749000371FC7CF0DB407FEFDCF11C11EBC8985B4
:1074A0009A85869D4001879D900C969D900C112495
:1074B000F10181A1E08CF18C26893789813021F49A
:1074C0002E153F0509F0B6C02E153F05B1F090E02E
:1074D000869D8001879D100D969D100D1124498574
:1074E0005A85489F9001499F300D589F300D1124B7
:1074F000A2016F817885C10166DCF101C1A0CC9C3D
:10750000F02D1124FD8BCA94612C712C2C2D30E0B0
:10751000388B2F87681479040CF088C0ED85FE85C0
:1075200084913196FE87ED8787FF7CC08F77DD24BD
:10753000D394D80ECC20F1F0F10121A130E0C301A9
:1075400069857A850E941D50289F7001299FF00C43
:10755000389FF00C11244F815885E40EF51E269FAC
:107560005001279FB00C369FB00C1124A40CB51C01
:10757000DB8639C0C30169857A850E941D50EF8082
:10758000F884E80EF91E5201A60EB71EF1CF0DB415
:1075900007FEFDCF0F8518890A0D1B1D2F85388921
:1075A0002E0D3F1DA501B701C10182DBCC2061F189
:1075B0008D898150F0F4F10181A190E0E80EF91E6F
:1075C00049855A85489F9001499F300D589F300D3D
:1075D00011246F817885260F371FE216F3061CF001
:1075E000A80EB91E7B017B8571507B877F3F79F6A2
:1075F00016C00DB407FEFDCF5B895EBD0DB407FE5E
:10760000FDCF69896EBDD5CF0DB407FEFDCF7B8957
:107610007EBD0DB407FEFDCF89898EBDCCCF6D0C2C
:10762000711C78CF8F5F680E711C74CF0DB407FE8C
:10763000FDCF45C08201060D171D015011092F8194
:10764000388589859A85280F391F21503109A20173
:107650006F817885C1012CDB181419040CF02CC043
:107660002D853E852F5F3F4FED85FE85849187FFF9
:1076700009C08F778F5F90E0881A990AF1014689D7
:10768000578907C08F5F90E0881A990AF101408DF1
:10769000518D009771F05EBD02D001D001C00895F8
:1076A00000004EBD0096009601D001C008950197DC
:1076B00091F73E872D87D0CF0DB407FEFDCF809187
:1076C0000B01816080930B01F10121A149855A854D
:1076D000249FC001259F900D112466960FB6F89443
:1076E000DEBF0FBECDBFDF91CF911F910F91FF90F5
:1076F000EF90DF90CF90BF90AF909F908F907F9052
:107700006F905F904F903F902F9008950F931F932D
:10771000CF93DF93DC01462F6D3009F478C090964B
:107720000C91909770E0023051F4FB01EA5FF64D46
:10773000849190E00696887FE0E1F0E01BC085E050
:10774000089F90011124F901EE59F54D859194910E
:10775000FB01B097E80FF91F8491F901EC59F54D41
:10776000E491013019F090E0F0E004C0E8E0F0E0CE
:1077700086E090E09196CC919197D0E0EC9F9001BB
:10778000ED9F300DFC9F300D11241A96ED91FC9168
:107790001B974A3059F42E0F3F1F1B963C932E9394
:1077A0001A9719961C921E92189731C094964C9174
:1077B00094974423F1F08C9FA0018D9F500D9C9FC6
:1077C000500D112418968D919C911997840F951F37
:1077D00052964D915C9153978417950750F02E0F58
:1077E0003F1F1B963C932E931A9719961C921E923C
:1077F0001897ED0110E02A853B8548855985CD0114
:107800001ADB28853985820F931F9987888781E045
:1078100090E0DF91CF911F910F91089590E0FC01CE
:107820003197E231F10508F04EC08827EC56FF4F42
:107830008F4F0C943050809180008F7703C08091DF
:1078400080008F7D80938000089580918000877FE5
:10785000F9CF84B58F7702C084B58F7D84BD08953C
:107860008091B0008F7703C08091B0008F7D8093AE
:10787000B0000895809190008F7707C080919000AC
:107880008F7D03C080919000877F80939000089542
:107890008091A0008F7707C08091A0008F7D03C0EA
:1078A0008091A000877F8093A0000895809120019F
:1078B0008F7707C0809120018F7D03C080912001C8
:1078C000877F8093200108953FB7F89480910B0C37
:1078D00090910C0CA0910D0CB0910E0C26B5A89BAC
:1078E00005C02F3F19F00196A11DB11D3FBFBA2F52
:1078F000A92F982F8827820F911DA11DB11DBC01B2
:10790000CD0142E0660F771F881F991F4A95D1F776
:107910000895CF93DF93282F30E0F901E85BFF4C07
:107920008491F901E351F54DD491F901E955F54DF3
:10793000C491CC2389F0811171DFEC2FF0E0EE0FC0
:10794000FF1FEA5BF54DA591B491EC91ED2381E029
:1079500090E021F480E002C080E090E0DF91CF91E0
:1079600008951F93CF93DF93282F30E0F901E85B50
:10797000FF4C8491F901E351F54DD491F901E9559A
:10798000F54DC491CC23C1F0162F811147DFEC2FA8
:10799000F0E0EE0FFF1FE357F54DA591B4918FB7BF
:1079A000F894111105C09C91ED2FE095E92302C0D8
:1079B000EC91ED2BEC938FBFDF91CF911F91089548
:1079C000CF93DF9390E0FC01E351F54D2491FC014E
:1079D000E955F54D8491882361F190E0880F991F56
:1079E000FC01E25DFF4CC591D491FC01E357F54DDC
:1079F000A591B491611109C09FB7F8948881209531
:107A000082238883EC912E230BC0623061F49FB7F0
:107A1000F8943881822F809583238883EC912E2BD4
:107A20002C939FBF06C08FB7F894E8812E2B288334
:107A30008FBFDF91CF910895863308F086539091E0
:107A40007B00282F2870977F922B90937B00877064
:107A5000806480937C0080917A00806480937A00B7
:107A600080917A0086FDFCCF80917800209179008A
:107A700090E0922B08954F925F926F927F928F9237
:107A80009F92BF92CF92DF92EF92FF920F931F933C
:107A9000CF93DF9300D000D0CDB7DEB760E0809108
:107AA00084088EDF60E0809185088ADF61E0809144
:107AB000870886DF61E08091860882DF80919208E6
:107AC000E0918A08F0918B089081892B80839091B6
:107AD0009308E0918E08F0918F088081282F30E084
:107AE000892F90E0809590958223932380838091C5
:107AF0008408A2DF8C01809184089EDF9801281BF6
:107B0000390B2C5F3F4F2930310548F4A801480F4D
:107B1000591FCA0195958795BB24B39401C0B12C18
:107B20000FEF13E0081B190B60E08091870848DF16
:107B300060E08091860844DF61E08091840840DF46
:107B400061E0809185083CDF90919508E091900874
:107B5000F09191088081282F30E0892F90E0809566
:107B6000909582239323808380919408E0918C08E0
:107B7000F0918D089081892B8083809186085CDF4D
:107B80007C018091860858DFA701481B590B4C5F88
:107B90005F4F4930510538F49701280F391FC9014B
:107BA0009595879501C0B12C4FEF53E07A01E81A03
:107BB000F90A61E08091870803DF60E08091840822
:107BC000FFDE90919208E0918A08F0918B08808105
:107BD000282F30E0892F90E0809590958223932381
:107BE000808380919508E0919008F09191089081B0
:107BF000892B8083809186081FDF6C018091840827
:107C00001BDF80908808909089088114910409F402
:107C10003FC0BC01990F880B990B0E94A64D2B0108
:107C20003C01B601DD0C880B990B0E94A64D9B010F
:107C3000AC01C301B2010E94754F20E030E040E882
:107C40005FE30E94104F2B013C01B801012E000C94
:107C5000880B990B0E94A64D9B01AC01C301B20198
:107C60000E94054E2B013C01B40180E090E00E948F
:107C7000A44D9B01AC01C301B2010E94054E20E05E
:107C800030E040E85AE30E94054E0E94DD4F05C0F7
:107C9000B601681B790B61507C4FB11002C060E0E7
:107CA00070E01A830983FC82EB827E836D83202F30
:107CB0003A814E2D5C817E8180E090E026960FB661
:107CC000F894DEBF0FBECDBFDF91CF911F910F9112
:107CD000FF90EF90DF90CF90BF909F908F907F901C
:107CE0006F905F904F9008958F929F92AF92BF9246
:107CF000CF92DF92EF92FF926B017C01E5DD4B01A9
:107D00005C01C114D104E104F104E9F0DDDDDC0122
:107D1000CB0188199909AA09BB09883E9340A1059E
:107D2000B10578F321E0C21AD108E108F10888EE24
:107D3000880E83E0981EA11CB11CC114D104E1047B
:107D4000F10421F7DECFFF90EF90DF90CF90BF904E
:107D5000AF909F908F9008952FB7F8946091070C83
:107D60007091080C8091090C90910A0C2FBF089516
:107D70000F931F93F1DF6093CD077093CE0780932D
:107D8000CF079093D007E091C507F091C607028412
:107D9000F385E02D85EC97E0199597FF1EC0DCDF99
:107DA0000091CD071091CE072091CF073091D007D9
:107DB000DC01CB01801B910BA20BB30B0091C90717
:107DC0001091CA072091CB073091CC0780179107FB
:107DD000A207B307C0F28FEF9FEF1F910F91089595
:107DE0001F920F920FB60F9211242F933F938F93F0
:107DF0009F93AF93BF938091070C9091080CA09133
:107E0000090CB0910A0C3091060C23E0230F2D379A
:107E100020F40196A11DB11D05C026E8230F02968E
:107E2000A11DB11D2093060C8093070C9093080CA4
:107E3000A093090CB0930A0C80910B0C90910C0C40
:107E4000A0910D0CB0910E0C0196A11DB11D809357
:107E50000B0C90930C0CA0930D0CB0930E0CBF91D7
:107E6000AF919F918F913F912F910F900FBE0F90E7
:107E70001F901895CF93DF93CDB7DEB7C154D109CA
:107E80000FB6F894DEBF0FBECDBF789484B5826084
:107E900084BD84B5816084BD85B5826085BD85B5AE
:107EA000816085BD80916E00816080936E0010922C
:107EB00081008091810082608093810080918100A7
:107EC0008160809381008091800081608093800038
:107ED0008091B10084608093B1008091B000816096
:107EE0008093B00080919100826080939100809196
:107EF00091008160809391008091900081608093D7
:107F000090008091A10082608093A1008091A100E7
:107F100081608093A1008091A00081608093A00087
:107F200080912101826080932101809121018160F3
:107F300080932101809120018160809320018091B4
:107F40007A00846080937A0080917A0082608093C6
:107F50007A0080917A00816080937A0080917A0023
:107F6000806880937A001092C10080E197E2A0E0DF
:107F7000B0E08093C8089093C908A093CA08B09352
:107F8000CB088DEC9BE19093C6088093C50881E0F7
:107F90008093C70840E457E76BE170E04093BD0869
:107FA0005093BE086093BF087093C00820ED3CE179
:107FB0003093BB082093BA088093BC088093AA072B
:107FC00061E082E0FDDC61E082E0CBDC61E083E047
:107FD000F7DC61E083E0C5DC61E084E0F1DC61E0D6
:107FE00084E0BFDC61E085E0EBDC61E085E0B9DCEA
:107FF00062E089E0E5DC1092B5071092B6071092B6
:10800000B7071092B8078CE291E0A0E0B0E080934F
:10801000B1079093B207A093B307B093B40782E07F
:1080200090E09093B0078093AF0796DE6093AB0724
:108030007093AC078093AD079093AE07E091D5079E
:10804000F091D60782E08083E091D107F091D207CA
:108050001082E091D307F091D4078FEC80831092C7
:10806000DD07E091D907F091DA0786E08083E0919F
:10807000D707F091D807808180618083E091D7078E
:10808000F091D807808188608083E091D707F091D4
:10809000D807808180688083E091D707F091D80766
:1080A00080818F7D808362E08091FA0889DC54DED4
:1080B000DC01CB01805D9740A109B1098093FE08E6
:1080C0009093FF08A0930009B093010987E3809380
:1080D00007091FB7F8948091B907811123C0ECED0F
:1080E000FAE28491E2E2FBE29491E82FF0E0EE0FF5
:1080F000FF1FE25DFF4CA591B491EC91E92319F4C7
:1081000061E085E32EDC61E085E35ADC8CB58061BB
:108110008CBD8CB580648CBD61E084E351DC61E092
:1081200083E34EDC8091B9078F5F8093B9071FBF4F
:108130008CB58093D7088CB58C7F8CBD8DB5816054
:108140008DBD8CB58F7D8CBD8CB5837F8CBD8CB582
:108150008093D60861E088E004DC65E070E080E0B0
:1081600090E0C2DD60E088E0FCDB64E170E080E08C
:1081700090E0BADD61E088E0F4DB66E970E080E081
:1081800090E0B2DDE6E4F2E0F49007E412E0FF20D4
:1081900009F434C0F80184910E94FA245801F2E0F5
:1081A000AF0EB11CF80131960491202F2078E22EF9
:1081B0000F776501102F115040F0F60184910E9455
:1081C000E924FFEFCF1ADF0AF6CF6501C00ED11CFC
:1081D0008601EE2089F02FEFC21AD20AF8016491CD
:1081E0006F3F21F070E080E090E004C064EF71E048
:1081F00080E090E079DD8601FA94C9CF81E0809338
:10820000F30886E30E94FA248091F30890E0883016
:10821000910570F5FC018827EE58FF4F8F4F0C94A5
:10822000305088E40BC088E215C088E807C088EEAB
:1082300011C088EC03C088E60DC088E00E94E924E4
:1082400080EF90E09093E3088093E20880E491E06F
:108250000BC088EA0E94E92480E491E09093E3084F
:108260008093E20880EF90E09093E5088093E40823
:1082700080910B018D7F80930B0180910B018E7F8C
:1082800080930B018AE28EBD00960096009601D085
:1082900001C0089580910B01826080930B011EBC88
:1082A00000000096009601D001C008951092EF08DA
:1082B0001092EE081EBC0000009601D001C0089587
:1082C0008091E2089091E30801979093DD088093F4
:1082D000DC089EBD00960096009601D001C008956E
:1082E0008EBD00000096009601D001C008958091D7
:1082F0000B018D7F80930B018BE28EBD0096009663
:10830000009601D001C0089580910B018260809396
:108310000B011EBC00000096009601D001C008951C
:108320001092ED081092EC081EBC0000009601D0DF
:1083300001C008958091E4089091E5080197909319
:10834000DF088093DE089EBD00960096009601D05F
:1083500001C008958EBD00000096009601D001C0B6
:10836000089580910B01816080930B018FEF9FEF47
:108370009093ED088093EC089093EF088093EE08BB
:108380009093DD088093DC089093DF088093DE08EB
:108390000E9465230E94BD1C63E872E0CE01019635
:1083A0000E94CD32CE0101960E942519CE01019680
:1083B0000E94AF326BE972E0CE0101960E94CD328D
:1083C000CE0101960E942519CE0101960E94AF327E
:1083D00065EA77E0CE0101960E94CD32CE0101968A
:1083E0000E942519CE0101960E94AF326AEF70E01B
:1083F00080E090E079DC6AEA72E0CE0101960E94AA
:10840000CD32CE0101960E942519CE0101960E941F
:10841000AF3269EC72E0CE0101960E94CD32CE01FE
:1084200001960E942519CE0101960E94AF326FEF8E
:1084300072E0CE0101960E94CD32CE0101960E94DB
:108440002519CE0101960E94AF3260E086E3B8DACA
:1084500011E01093020266E381EB98E00E94A823EA
:10846000811111C06BE273E0CE0101960E94CD3202
:10847000CE0101960E942519CE0101960E94AF32CD
:108480001092A90725C06DE473E0CE0182960E9488
:10849000CD3281EB98E00E94F32E60E170E0CE01D6
:1084A00082960E94F331BE016E5D7F4FCE01019630
:1084B0000E94B432CE0101960E942519CE01019688
:1084C0000E94AF321093A907CE0182960E94AF326C
:1084D00067E388EA98E00E94A823811111C069E748
:1084E00073E0CE0101960E94CD32CE0101960E942A
:1084F0002519CE0101960E94AF321092A80726C01E
:108500006BE973E0CE0182960E94CD3288EA98E052
:108510000E94F32E60E170E0CE0182960E94F3315A
:10852000BE016E5D7F4FCE0101960E94B432CE0136
:1085300001960E942519CE0101960E94AF3281E07A
:108540008093A807CE0182960E94AF3268E38FE93C
:1085500098E00E94A823811111C067EC73E0CE015E
:1085600001960E94CD32CE0101960E942519CE01BE
:1085700001960E94AF321092A70726C069EE73E001
:10858000CE0182960E94CD328FE998E00E94F32EB0
:1085900060E170E0CE0182960E94F331BE016E5D13
:1085A0007F4FCE0101960E94B432CE0101960E9407
:1085B0002519CE0101960E94AF3281E08093A70772
:1085C000CE0182960E94AF3269E386E998E00E946C
:1085D000A823811111C065E174E0CE0101960E94CB
:1085E000CD32CE0101960E942519CE0101960E943E
:1085F000AF321092A60726C067E374E0CE018296E0
:108600000E94CD3286E998E00E94F32E60E170E08E
:10861000CE0182960E94F331BE016E5D7F4FCE0186
:1086200001960E94B432CE0101960E942519CE0116
:1086300001960E94AF3281E08093A607CE01829618
:108640000E94AF321092AA0780E090E00E9465235A
:10865000EE24EA94FE2C04E110E020EA30E040E051
:1086600050E060E070E080ED98E00E94E33682E048
:1086700090E09093D9088093D8089093DB0880937A
:10868000DA0884E08093F0081092E9081092E80874
:108690001092E7081092E60863E674E0CE010196B6
:1086A0000E94CD3222E030E042E050E062E070E033
:1086B00089819A810E94252210920202CE010196A0
:1086C0000E94AF32D8D92CAB3DAB4EAB5FAB68AF9D
:1086D00079AF2CA93DA9AEA8BFA808AD19AD80916E
:1086E000820890918308801791070CF0CAC2C0904D
:1086F000E408D090E5080D2C000CEE08FF08C90135
:10870000330FAA0BBB0B9C01AD0124563109410963
:10871000510966277727CB016C197D098E099F09BE
:108720000E940E5020E233E040E050E00E94B94E3B
:10873000C20ED31EE41EF51EDBAECAAE8090E20868
:108740009090E3082401990C66087708C501BB0CDA
:10875000AA0BBB0B9C01AD012659310941095109F6
:1087600066277727CB0164197509860997090E9446
:108770000E502EEE32E040E050E00E94B94E49012A
:108780005A01840C951CA61CB71C80E794E00E943B
:10879000942630E4432E5524539448185908C201B6
:1087A0000E94212785E794E00E949426C6010E943A
:1087B00021278BE794E00E949426C8010E940C2791
:1087C000F3E3CF1AD1082FE4C216D10408F0FBC09E
:1087D0008091BA079091BB07019709F0F4C086E336
:1087E00091E08819990997FD05C090931402809330
:1087F000130204C01092140210921302809113020B
:10880000909114028931914034F088E191E0909385
:10881000140280931302A0911302B091140226EE69
:1088200030E00E94385028E131E040E050E00E9402
:10883000B94E69017A0189E1C80ED11CE11CF11C15
:10884000860161E086E0BCD8C114D104E104F104E2
:1088500011F460E007C09FEFC916D104E104F104F0
:1088600021F461E086E07DD8ACC0EEE4F0E38491D1
:1088700090E0FC013197E231F10508F09DC08827B6
:10888000E658FF4F8F4F0C94305084B5806884BDFC
:10889000C7BC97C084B5806284BDC8BC92C08091BB
:1088A0008000806880938000D0928900C092880008
:1088B00088C080918000806280938000D0928B007D
:1088C000C0928A007EC08091800088608093800082
:1088D000D0928D00C0928C0074C08091B0008068EE
:1088E0008093B000C092B3006CC08091B0008062F1
:1088F0008093B000C092B40064C080919000806802
:1089000080939000D0929900C09298005AC08091B4
:108910009000806280939000D0929B00C0929A0059
:1089200050C080919000886080939000D0929D000C
:10893000C0929C0046C08091A00080688093A000F7
:108940008091A0008F7B8093A000D092A900C0925C
:10895000A80037C08091A00080628093A000D092D0
:10896000AB00C092AA002DC08091A00088608093C7
:10897000A000D092AD00C092AC0023C08091200135
:10898000806880932001D0922901C092280119C0EB
:1089900080912001806280932001D0922B01C092AF
:1089A0002A010FC080912001886080932001D0921D
:1089B0002D01C0922C0105C0003811050CF051CFDB
:1089C00048CF0E940E258091BA079091BB0703976C
:1089D00009F00FC1209003023090040200910502BB
:1089E00010910602E0900702F090080244D82AA3F2
:1089F0003BA34CA35DA36EA37FA32AA13BA1CCA064
:108A0000DDA04EA15FA15DAF4CAF80918208909137
:108A10008308841795070CF0ECC08090E4089090D0
:108A2000E508092C000CAA08BB08C901330FAA0BE2
:108A3000BB0B9C01AD012456310941095109662740
:108A40007727CB01681979098A099B090E940E5082
:108A500020E233E040E050E00E94B94EDA01C90163
:108A6000880D991DAA1DBB1D22968CAF9DAFAEAF80
:108A7000BFAF22976EAC7FAC2091E2083091E30843
:108A80004901330FAA08BB0880E794E00E949426AE
:108A9000C601DD0CAA0BBB0B9C01AD0126593109A7
:108AA0004109510966277727CB01681979098A0995
:108AB0009B090E940E502EEE32E040E050E00E94F2
:108AC000B94EDA01C901880D991DAA1DBB1D20E40C
:108AD000C22EDD24D394C81AD90AC6010E942127C8
:108AE00085E794E00E9494268EAD9FAD0E942127D9
:108AF0008BE794E00E9494268CAD9DAD0E940C27DC
:108B0000C1018B5B9F4F8C159D050CF072C089963F
:108B10008C159D050CF46DC068019FE0C90ED11C39
:108B2000C614D704FCF0C801449768167906D4F03F
:108B300080910B0290910C02E816F9069CF480914A
:108B400007029091080244969093080280930702CE
:108B500065EA77E0CE0101960E94CD32B7016C5EE6
:108B60007F4F24C0C8010E96861597050CF041C0B2
:108B70000E5C1F4F06151705E4F1809109029091D4
:108B80000A028E159F05ACF58091070290910802AC
:108B90004497909308028093070265EA77E0CE013C
:108BA00001960E94CD32B70164517109CE01019640
:108BB0000E94F33168E874E0CE0101960E942232EF
:108BC000EE24EA94FE2C09E110E026E430E0A60150
:108BD000B10180ED98E00E94E33624E030E0A60188
:108BE000B10189819A810E942522CE0101960E94BD
:108BF000AF32A0EA4A1651049CF4EAADFBADE2386C
:108C0000F1052CF58091BA079091BB07892BA1F54E
:108C1000CC24C394D12CD092BB07C092BA0729C0F0
:108C200020EA4216510469F14AAD5BAD4238510564
:108C30000CF0CCC28091BA079091BB07892BE1F46C
:108C400082E090E09093BB078093BA0712C08AAD90
:108C50009BAD83389105ACF08091BA079091BB072A
:108C6000009709F099C2A3E0B0E0B093BB07A093CE
:108C7000BA0781E0809302026AEF70E080E090E042
:108C800033D8C090C808D090C908E090CA08F090C6
:108C9000CB0862D80091CC081091CD082091CE0865
:108CA0003091CF080C0D1D1D2E1D3F1D680179014F
:108CB000C61AD70AE80AF90AD701C6018A3F910500
:108CC000A105B10538F48091BA079091BB070297CE
:108CD00009F4BCC280910202882309F4CDC18091BD
:108CE000BA079091BB070097F1F570EEE72EFF24CD
:108CF000FA940AE814E02EE630E040EA50E064E13D
:108D000070E080E090E00E94CA18E0EEEE2EE7E00E
:108D1000FE2E01E914E02EE630E040EA50E064E186
:108D200070E080EA90E00E94CA18FFE1EF2EF12C7B
:108D300007E914E02EE630E040EA50E062E870E037
:108D400080E090E00E94CA18809100029091010298
:108D5000E12CA8EFFA2E892B19F00FE914E02CC0B2
:108D600004EA14E029C08130910589F540EEE42E33
:108D700047E0F42E0AEA14E02EE630E040EA50E044
:108D800062E870E080E090E00E94CA18E12C58EFA1
:108D9000F52E00EB14E02EE630E040E451E064E113
:108DA00070E080E090E00E94CA180E940E256FE1FA
:108DB000E62EF12C0BEB14E02EE630E040EA50E01A
:108DC00062E870E080EA90E00E94CA18E0C0029772
:108DD00009F0DDC0EE24EA94FE2C05EA17E02CED44
:108DE00030E040E451E064E170E080E090E00E9417
:108DF000CA180E949F244B015C0180E00E940B2452
:108E000081E00E940B246B017C0165E676E0CE01D7
:108E10008E960E94CD32B501A401CE018E960E949D
:108E2000933168E874E0CE018E960E942232BE0132
:108E3000625D7F4FCE0101960E94B43224E030E0A3
:108E40004EE150E062E070E089819A810E94252223
:108E5000CE0101960E94AF3263E776E0CE018E9696
:108E60000E949A32B701A601CE018E960E949331DC
:108E700060EC74E0CE018E960E942232BE01625DEB
:108E80007F4FCE0101960E94B43224E030E045E3EA
:108E900050E062E070E089819A810E942522CE0133
:108EA00001960E94AF32C090BD08D090BE08E090FD
:108EB000BF08F090C0080E94AC3E0091C10810911C
:108EC000C2082091C3083091C4080C0D1D1D2E1D31
:108ED0003F1D68017901C61AD70AE80AF90AC701D5
:108EE000B60120E63AEE40E050E069D7CA01B90188
:108EF0006F5F7F4F8F4F9F4F19A618A61BA61AA60C
:108F00001DA61CA62AE0AE014F5F5F4F6AD3BE01CB
:108F10006F5F7F4FCE0188960E949A32BE01685DD6
:108F20007F4FCE018E960E943032CE0188960E94ED
:108F3000AF3269EC74E0CE018E960E942232BE01FF
:108F4000625D7F4FCE0101960E94B43224E030E092
:108F50004CE450E062E070E089819A810E94252211
:108F6000CE0101960E94AF323FE1E32EF12C0BEBD4
:108F700014E02EE630E040EA50E062E870E080EA7B
:108F800090E00E94CA18CE018E960E94AF32809166
:108F9000BA079091BB07039709F06CC0EE24EA94DE
:108FA000FE2C05EA17E02CED30E040E451E064E1EE
:108FB00070E080E090E00E94CA189FE1E92EF12C59
:108FC0000BEB14E02EE630E040EA50E062E870E09F
:108FD00080EA90E00E94CA18409003025090040278
:108FE000C0900502D090060220900702309008023F
:108FF000320129E6620E711C42014AE5840E911C81
:10900000B6016C5E7F4F52015BE4A50EB11C960168
:10901000255031097B018301A401C5010E9445252A
:10902000B601625E7F4F9601295C3F4F7B01A40130
:10903000C5010E94452565EA77E0CE0101960E94B0
:10904000CD32B101CE0101960E94F33168E874E09F
:10905000CE0101960E942232A601415F5F4F24E0BB
:1090600030E0B20189819A810E942522CE010196C9
:109070000E94AF321092020285EC97E00E947D2F91
:10908000181619060CF07BC065EA77E0CE01019650
:109090000E94CD320E94B83E97FD0CC088A719A649
:1090A00041E050E0BE01685D7F4FCE0101960E9415
:1090B0003631F0CF6EED74E0CE0188960E94CD324D
:1090C0004D815E8169817A81CE0188960E94363118
:1090D000811104C0CE0188960E946932BE01685D8C
:1090E0007F4FCE018E960E94B432CE0188960E94A8
:1090F000AF32CE0101960E94AF322AA93BA9263396
:10910000310530F125E330E040E050E0BE01625D22
:109110007F4FCE0101960E94E132CE0101960E945E
:109120002519CE0101960E94AF322AA93BA945E339
:1091300050E0BE01625D7F4FCE0101960E94E13298
:10914000BE016F5F7F4FCE018E960E943032D1CF2D
:109150002150310940E050E0BE01625D7F4FCE01F9
:1091600001960E94E132CE0101960E942519CE019E
:1091700001960E94AF32CE018E960E94AF320E94BD
:10918000AC3E85EC98E00E9480188AEB98E00E9443
:1091900080180E941A3096CA019709F06DCDE12C13
:1091A000F12C00EF10E020E431E040E050E060E01E
:1091B00070E080ED98E00E94E33661E089E00E9473
:1091C000E03C60E089E00E94B13C56CDAAADBBAD69
:1091D000A338B1050CF455CD8091BA079091BB0727
:1091E000009759F58091000290910102892B51F06E
:1091F0001092BC0881E0809302021092010210924A
:1092000000023ACD11E01093BC08E091BA08F09149
:10921000BB0819950E94AC3E6093C1087093C208C8
:109220008093C3089093C40810930202E1E0F0E039
:10923000F0930102E09300021FCD0197039708F01D
:109240001BCD1092BB071092BA0713CD81E080931B
:10925000020240CD80E798E00E94AF3286E798E0B6
:109260000E94AF328CE798E00C94AF32EF92FF92FD
:109270000F931F93CF93DF93E5ECF7E013821282F5
:1092800088EE93E0A0E0B0E084839583A683B78363
:1092900023E232E03183208325EC30E035872487D8
:1092A00024EC30E03787268720EC30E0318B208BB0
:1092B00021EC30E0338B228B22EC30E0358B248B99
:1092C00026EC30E0378B268B118E128E138E148E87
:1092D00004E618E0F8011382128284839583A68342
:1092E000B78385E392E091838083E2E6F8E080E54E
:1092F00080831182E8E0F9E01582168211861386D8
:1093000082E090E0A0E0B0E084879587A687B787E9
:1093100013A215A614A687E492E093A782A717A626
:10932000A5EFB8E080E215968C93159786E1169626
:109330008C931697EDE0FBE2E4911796EC93179768
:10934000E7ECFAE2E4911896EC93189740E85EE3B4
:1093500060E070E01D964D935D936D937C93509704
:10936000C0EDD8E01B821A8283E592E0998388835E
:1093700060E088E00E94B13C61E088E00E94E03C4F
:109380008BE0E82EFF24F394F701808182608083D4
:1093900061E080E30E94E03CF7018081816080838E
:1093A00061E081E30E94E03C80EF90E09B8B8A8B40
:1093B00080E491E09D8B8C8B1BA2198618861B86FE
:1093C0001A8621E028A329A38FEF9FEF9F8B8E8B16
:1093D000198E188E198A188A2CA31AA29D8F8C8F29
:1093E0009F8F8E8F9D878C879F878E8786ED90E0DD
:1093F0009B8F8A8FE5ECF8E0128211821082138233
:109400001482158216821782108611861286EAEB64
:10941000F8E0128211821082138214821582168261
:109420001782108611861286E1EBF8E01382128211
:109430008BE692E09183808316830583E8EAF8E067
:10944000138212829183808316830583EFE9F8E00B
:10945000138212829183808316830583E6E9F8E004
:10946000138212829183808316830583A2E8B8E079
:109470008AE312968C9312978BE314968C9314972D
:109480008EE113968C9313978FE115968C93159715
:109490008DE491E017969C938E931697E6ECFAE292
:1094A000E491F0E0EE0FFF1FE357F54D85919491A5
:1094B00019969C938E931897E1EEFAE2E491F0E00E
:1094C000EE0FFF1FE357F54D859194911B969C93EA
:1094D0008E931A97E2EEFAE2E491F0E0EE0FFF1FAE
:1094E000E357F54D859194911D969C938E931C970F
:1094F000E5ECFAE2E491F0E0EE0FFF1FE357F54DE3
:10950000859194911F969C938E931E97ECE0FBE2BD
:10951000E4915096EC935097E7E2FBE2E491529687
:10952000EC935297E8E2FBE2E4915196EC93519769
:10953000EBE0FBE2E4915396EC9353978AE090E0E2
:109540008D939C9365EA77E08CE798E00E94CD329A
:1095500065EA77E086E798E00E94CD3265EA77E039
:1095600080E798E0DF91CF911F910F91FF90EF90EE
:109570000C94CD32EF920F931F93CF93DF93E801BA
:1095800047FD02C034E001C034E1E42F440FFF0B7B
:10959000F7FF03C0F195E195F109E32E022F2E2F7D
:1095A000AE0159D0CE01DF91CF911F910F91EF9075
:1095B0000895BB274A3031F4992322F4BDE29095F7
:1095C00081959F4F30C0BB272A3051F4992342F434
:1095D000BDE290958095709561957F4F8F4F9F4F1D
:1095E00001C0BB27FA01A62F6217710581059105FD
:1095F000330B30FB66F0AA27660F771F881F991F71
:10960000AA1FA21710F0A21B63953850A9F7A05DFE
:10961000AA3308F0A95DA19336F7B111B193108276
:10962000CA017EC2BB27FB015527AA27880F991FB5
:10963000AA1FA41710F0A41B83955051B9F7A05D81
:10964000AA3308F0A95DA193009779F7B111B193FE
:109650001192CB0165C24F925F926F927F929F925F
:10966000AF92BF92CF92DF92EF92FF920F931F9330
:10967000CF93DF93CDB7DEB729970FB6F894DEBF4F
:109680000FBECDBF6A01122FB02E2BE3201720F0A2
:10969000FF24F394F00E02C0BCE3FB2E0F2D27E055
:1096A000AE014F5F5F4F64D1AC018981982F9970F3
:1096B000913031F0E1FC06C0E0FE06C090E205C04A
:1096C0009DE203C09BE201C090E0EE2DE07183FFBC
:1096D0003CC0911102C083E001C084E0811718F4FE
:1096E000212F281B01C020E0E1110BC0F601822FC1
:1096F00030E2882319F031938150FBCFC20ED11C88
:1097000020E0992329F0D6019C93F60131966F0150
:10971000C6010396E2FE0AC03EE4D6013C9341E452
:1097200011964C93119712963C9306C03EE6F601B3
:10973000308341E641833283FC01322F40E2332300
:1097400009F442C041933150FACF82FF44C09111D5
:1097500002C083E001C084E0811718F4212F281B88
:1097600001C020E0E1110BC0F601822F30E2882316
:1097700019F031938150FBCFC20ED11C20E0992308
:1097800029F0D6019C93F60131966F01C60103962C
:10979000E2FE0BC039E4D6013C933EE411963C93C3
:1097A000119736E412963C9307C039E6F6013083F0
:1097B0003EE6318336E63283FC01322F40E233232A
:1097C00019F041933150FBCFFC01E20FF11D1082E3
:1097D0008EEF9FEFB7C0F1E0911101C0F0E06F2F65
:1097E00070E01416150624F49A012F5F3F4F02C053
:1097F00021E030E0260F371FBB2029F06B2D70E0F1
:109800006F5F7F4F02C060E070E0260F371F612F4F
:1098100070E0261737071CF4121B212F01C020E02F
:109820003E2D387159F4D601322F60E2332319F0FE
:109830006D933150FBCFC20ED11C20E0FF2331F0DD
:10984000D6019C93B6016F5F7F4F6B01E1110BC096
:10985000F601922F30E3992319F031939150FBCF09
:10986000C20ED11C20E09F2D940F3A81782F707189
:10987000A72E84FF03C0313309F49150191624F444
:10988000993018F098E001C091E0E42F852F57FF40
:1098900002C0E0E080E06E2F782FE0E0F0E0AEE282
:1098A0009A2E3A01691A71082A01461A570A0B2D95
:1098B00010E01195019511096F3F8FEF780729F49A
:1098C000D6019C92C60101966C014617570784F099
:1098D000661677066CF47F01E40CF51CA1E0B0E09D
:1098E000AC0FBD1FEA0EFB1ED7011196BC9002C043
:1098F00090E3B92E615071093196C60101967C0141
:109900006017710724F0D601BC926C01D5CF6417A3
:10991000750741F4363320F4353321F4A11002C029
:1099200081E3B82EF601B082F701822F90E28823FE
:1099300019F091938150FBCFF701E20FF11D1082D6
:1099400080E090E029960FB6F894DEBF0FBECDBF41
:10995000DF91CF911F910F91FF90EF90DF90CF900B
:10996000BF90AF909F907F906F905F904F900895C1
:10997000283008F027E03327DA01990F311D87FDE1
:10998000916000966105710539F432602E5F3D9358
:1099900030E32A95E1F708959F3F30F08038710554
:1099A000610509F03C5F3C5F3D93913008F08068B1
:1099B000911DDF93CF931F930F93FF92EF92192F77
:1099C000987F9695E92F96959695E90FFF27EA558A
:1099D000FE4F99273327EE24FF24A701E7010590C6
:1099E0000894079428F4360FE71EF81E491F511DEE
:1099F000660F771F881F991F0694A1F7059007949B
:109A000028F4E70EF81E491F561FC11D770F881F47
:109A1000991F661F0694A1F70590079428F4F80E85
:109A2000491F561FC71FD11D880F991F661F771F1B
:109A30000694A1F70590079420F4490F561FC71FFD
:109A4000D81F990F661F771F881F0694A9F7849166
:109A50001095177041F0D695C79557954795F7948F
:109A6000E7941A95C1F7ECE4F1E06894159015912C
:109A700035916591959105907FE27395E118F10A12
:109A8000430B560BC90BD009C0F7E10CF11E431F65
:109A9000561FC91FD01D7EF4703311F48A95E6CF8E
:109AA000E894015030F0080F0AF40027021708F478
:109AB000202F2395022F7A3328F079E37D932A957E
:109AC000E9F710C07D932A9589F6069497956795D6
:109AD000379517951794E118F10A430B560BC90BEC
:109AE000D00998F023957E9173957A3308F070E34E
:109AF0007C932013B8F77E9170617D9330F083954D
:109B000071E37D9370E32A95E1F71124EF90FF90C4
:109B10000F911F91CF91DF91992787FD909508951F
:109B2000DC01FC01672F71917723E1F7329704C0C4
:109B30007C916D9370836291AE17BF07C8F308954F
:109B400040D008F481E00895E89409C097FB3EF402
:109B500090958095709561957F4F8F4F9F4F99237A
:109B6000A9F0F92F96E9BB279395F69587957795F8
:109B70006795B795F111F8CFFAF4BB0F11F460FFB8
:109B80001BC06F5F7F4F8F4F9F4F16C0882311F010
:109B900096E911C0772321F09EE8872F762F05C024
:109BA000662371F096E8862F70E060E02AF09A95BF
:109BB000660F771F881FDAF7880F9695879597F9B4
:109BC0000895990F0008550FAA0BE0E8FEEF16164E
:109BD0001706E807F907C0F012161306E407F507A1
:109BE00098F0621B730B840B950B39F40A2661F015
:109BF000232B242B252B21F408950A2609F4A140B8
:109C0000A6958FEF811D811D08950BD078C069D076
:109C100028F06ED018F0952309F05AC05FC01124C7
:109C2000A2C07ED0A0F3959FD1F3950F50E0551FB1
:109C3000629FF001729FBB27F00DB11D639FAA27A1
:109C4000F00DB11DAA1F649F6627B00DA11D661FF0
:109C5000829F2227B00DA11D621F739FB00DA11D11
:109C6000621F839FA00D611D221F749F3327A00DCB
:109C7000611D231F849F600D211D822F762F6A2F67
:109C800011249F5750408AF0E1F088234AF0EE0FEC
:109C9000FF1FBB1F661F771F881F91505040A9F7F9
:109CA0009E3F510570F014C05EC05F3FECF3983EDC
:109CB000DCF3869577956795B795F795E7959F5F60
:109CC000C1F7FE2B880F911D9695879597F90895FA
:109CD00097F99F6780E870E060E008959FEF80EC5F
:109CE000089500240A941616170618060906089502
:109CF00000240A9412161306140605060895092E68
:109D00000394000C11F4882352F0BB0F40F4BF2BD6
:109D100011F460FF04C06F5F7F4F8F4F9F4F089516
:109D200057FD9058440F551F59F05F3F71F047950C
:109D3000880F97FB991F61F09F3F79F087950895F1
:109D4000121613061406551FF2CF4695F1DF08C010
:109D5000161617061806991FF1CF8695710561052D
:109D600008940895E894BB2766277727CB0197F9D5
:109D70000895052E97FB16F400940FD057FD05D0DB
:109D80001ED007FC02D046F408C05095409530958F
:109D900021953F4F4F4F5F4F089590958095709557
:109DA00061957F4F8F4F9F4F08952BD0A59F900DAA
:109DB000B49F900DA49F800D911D11240895A1E2E0
:109DC0001A2EAA1BBB1BFD010DC0AA1FBB1FEE1F35
:109DD000FF1FA217B307E407F50720F0A21BB30B80
:109DE000E40BF50B661F771F881F991F1A9469F7FC
:109DF00060957095809590959B01AC01BD01CF0158
:109E00000895A29FB001B39FC001A39F700D811D53
:109E10001124911DB29F700D811D1124911D089573
:109E20005058BB27AA270ED06ACF5BDF30F060DF27
:109E300020F031F49F3F11F41EF450CF0EF4E09562
:109E4000E7FB46CFE92F6CDF80F3BA176207730791
:109E50008407950718F071F49EF584CF0EF4E09511
:109E60000B2EBA2FA02D0B01B90190010C01CA01D4
:109E7000A0011124FF27591B99F0593F50F4503E7F
:109E800068F11A16F040A22F232F342F4427585F71
:109E9000F3CF469537952795A795F0405395C9F789
:109EA0007EF41F16BA0B620B730B840BBAF0915041
:109EB000A1F0FF0FBB1F661F771F881FC2F70EC0E0
:109EC000BA0F621F731F841F48F4879577956795B3
:109ED000B795F7959E3F08F0B3CF9395880F08F09C
:109EE0009927EE0F9795879508950CD008CF00DF3E
:109EF00040F0F7DE30F021F45F3F19F0E9CE511168
:109F000032CFECCE0DDF98F39923C9F35523B1F38B
:109F1000951B550BBB27AA2762177307840738F0D8
:109F20009F5F5F4F220F331F441FAA1FA9F333D037
:109F30000E2E3AF0E0E830D091505040E695001CEB
:109F4000CAF729D0FE2F27D0660F771F881FBB1FA7
:109F5000261737074807AB07B0E809F0BB0B802D81
:109F6000BF01FF2793585F4F2AF09E3F510568F0CD
:109F7000AFCEF9CE5F3FECF3983EDCF38695779554
:109F80006795B795F7959F5FC9F7880F911D9695CF
:109F9000879597F90895E1E0660F771F881FBB1F2B
:109FA000621773078407BA0720F0621B730B840BD8
:109FB000BA0BEE1F88F7E095089504D06894B111AC
:109FC000D2CE0895B5DE88F09F5790F0B92F99272B
:109FD000B751A0F0D1F0660F771F881F991F1AF0B4
:109FE000BA95C9F712C0B13081F0BCDEB1E0089576
:109FF000B9CE672F782F8827B85F39F0B93FCCF3F7
:10A00000869577956795B395D9F73EF490958095A9
:10A01000709561957F4F8F4F9F4F0895DB018F9310
:10A020009F93C3DEBF91AF91A29F800D911DA39F0F
:10A03000900DB29F900D1124089597FB072E16F4F2
:10A04000009406D077FD08D019D007FC05D03EF467
:10A05000909581959F4F0895709561957F4F0895D4
:10A06000EE0FFF1F881F8BBF0790F691E02D19940C
:10A07000C8DEB7FF0895821B930B0895AA1BBB1B74
:10A0800051E107C0AA1FBB1FA617B70710F0A61BF8
:10A09000B70B881F991F5A95A9F780959095BC0119
:10A0A000CD010895CF93DF938230910510F482E0C3
:10A0B00090E0E091110CF091120C20E030E0C0E053
:10A0C000D0E0309711F14081518148175907C0F015
:10A0D0004817590761F482819381209719F09B8377
:10A0E0008A832BC09093120C8093110C26C02115EB
:10A0F000310519F04217530718F49A01BE01DF0128
:10A10000EF010280F381E02DDCCF2115310509F14B
:10A11000281B390B2430310590F412968D919C91B7
:10A1200013976115710521F0FB019383828304C0AD
:10A130009093120C8093110CFD01329644C0FD01E6
:10A14000E20FF31F81939193225031092D933C9399
:10A150003AC020910F0C3091100C232B41F4209128
:10A160001B0230911C023093100C20930F0C209195
:10A17000190230911A022115310541F42DB73EB76D
:10A1800040911D0250911E02241B350BE0910F0CD3
:10A19000F091100CE217F307A0F42E1B3F0B2817C9
:10A1A000390778F0AC014E5F5F4F2417350748F050
:10A1B0004E0F5F1F5093100C40930F0C819391939F
:10A1C00002C0E0E0F0E0CF01DF91CF9108950F935E
:10A1D0001F93CF93DF93009709F48CC0FC01329753
:10A1E000138212820091110C1091120C01151105AD
:10A1F00081F420813181820F931F20910F0C3091C7
:10A20000100C2817390779F5F093100CE0930F0C18
:10A2100071C0D80140E050E0AE17BF0750F412966D
:10A220002D913C911397AD012115310509F1D9010B
:10A23000F3CF9D01DA013383228360817181860F20
:10A24000971F8217930769F4EC0128813981260F43
:10A25000371F2E5F3F4F318320838A819B819383F9
:10A260008283452B29F4F093120CE093110C42C029
:10A270001396FC93EE931297ED01499159919E012B
:10A28000240F351FE217F30771F480819181840F49
:10A29000951F029611969C938E93828193811396BB
:10A2A0009C938E931297E0E0F0E0D80112968D9186
:10A2B0009C911397009719F0F8018C01F6CF8D91BE
:10A2C0009C9198012E5F3F4F820F931F20910F0C9E
:10A2D0003091100C2817390769F4309729F410923F
:10A2E000120C1092110C02C0138212821093100CE7
:10A2F00000930F0CDF91CF911F910F9108956F92F2
:10A300007F928F929F92AF92BF92CF92DF92EF9205
:10A31000FF920F931F93CF93DF93EC01009781F48B
:10A32000CB01DF91CF911F910F91FF90EF90DF90C4
:10A33000CF90BF90AF909F908F907F906F90B2CE54
:10A34000FC01E60FF71F9C0122503109E217F307C9
:10A3500008F4A8C0D9010D911C9111970617170791
:10A36000A8F00530110508F49BC0C80104978617B2
:10A37000970708F495C002501109061B170B0193AB
:10A3800011936D937C93CF0122DF8AC05B01A01AE9
:10A39000B10A4C01800E911EA091110CB091120CCB
:10A3A00040E050E0E12CF12C109709F44AC0A815C8
:10A3B000B905D1F56D907C901197630182E0C80ECC
:10A3C000D11CCA14DB0480F1A3014A195B096A019C
:10A3D00082E0C80ED11C1296BC9012971396AC91D5
:10A3E000B5E0CB16D10440F0B282A3835183408301
:10A3F000D9016D937C930AC00E5F1F4FC301800F7C
:10A40000911FF90191838083EB2DFA2FE114F10460
:10A4100031F0D7011396FC93EE93129741C0F0935D
:10A42000120CE093110C3CC08D919C911197481730
:10A43000590708F4AC017D0112960D90BC91A02D36
:10A44000B3CF80910F0C9091100C88159905E1F411
:10A4500046175707C8F48091190290911A02009785
:10A4600041F48DB79EB740911D0250911E02841B8E
:10A47000950BE817F907B0F4F093100CE0930F0C6C
:10A48000F901718360830CC0CB010CDE7C01009765
:10A4900049F0A801BE011BD0CE0199DEC70104C05E
:10A4A000CE0102C080E090E0DF91CF911F910F912B
:10A4B000FF90EF90DF90CF90BF90AF909F908F90E4
:10A4C0007F906F90089581E090E0F89410C0FB01B8
:10A4D000DC0102C001900D9241505040D8F7089520
:10A4E000FB01DC0101900D920020E1F7089518E1D5
:10A4F000C8E4D8E100E005C0802FFE01B1DD21965F
:10A50000011DC934D10780E00807B1F7F894FFCFE7
:10A51000010001C8001E00640014002C010A005A4A
:10A52000002C011801FFFFFFFF0000130C8000004A
:10A53000000000B32F212F4C2FF92F7D2F5B2F6FA1
:10A540002F00000000DF30B0307D188430A8309438
:10A5500030853000000000922B212F7D187C1800E0
:10A56000000000863B212F7D187C18000000000DA4
:10A5700031212F7D187C18000000009F35212F7D90
:10A58000187C1854277F2E322768350001020300FB
:10A59000010203426F6F74696E6720477265656ED2
:10A5A000686F7573654F532E2E2E00566572736952
:10A5B0006F6E3A20302E322E32005B4641494C45B8
:10A5C000445D2053442043617264206E6F742064A4
:10A5D0006574656374656421005B20204F4B202007
:10A5E0005D20456E61626C696E6720706F77657281
:10A5F000736176696E672066656174757265732E26
:10A600002E2E202020202020202020202020005B13
:10A610004641494C45445D20506F776572736176C1
:10A62000696E673A20417267756D656E74206D754D
:10A630007374206265203E20302E005B20494E4618
:10A640004F205D20536F696C2073656E736F7220AD
:10A650003120756E706C75676765642E005B202015
:10A660004F4B20205D20536F696C2073656E736FB4
:10A6700072203120636F6E6E65637465642E2056A0
:10A68000657273696F6E3A20005B20494E464F2019
:10A690005D20536F696C2073656E736F722032207A
:10A6A000756E706C75676765642E005B20204F4B7C
:10A6B00020205D20536F696C2073656E736F72206C
:10A6C0003220636F6E6E65637465642E205665720A
:10A6D00073696F6E3A20005B20494E464F205D2023
:10A6E000536F696C2073656E736F72203320756EC3
:10A6F000706C75676765642E005B20204F4B2020CF
:10A700005D20536F696C2073656E736F7220332008
:10A71000636F6E6E65637465642E2056657273692F
:10A720006F6E3A20005B20494E464F205D20536FEC
:10A73000696C2073656E736F72203420756E706C57
:10A7400075676765642E005B20204F4B20205D20DD
:10A75000536F696C2073656E736F72203420636F62
:10A760006E6E65637465642E2056657273696F6ED4
:10A770003A20005761746572204C6576656C3A002A
:10A7800058203D20000959203D2000095072657372
:10A7900073757265203D2000250053797374656DD3
:10A7A000005374617473004F7074696F6E7300535B
:10A7B000746F700053746172740052657365740035
:10A7C0004272696768746E657373004261636B00FF
:10A7D000206465677265657300206D696E757465C8
:10A7E0007320756E74696C207761746572005365AF
:10A7F0007269616C3A20005B20204F4B20205D2065
:10A80000536F696C2073656E736F722034207465AA
:10A810006D70657261747572653A200020432C205A
:10A82000002046005B20204F4B20205D20536F69A5
:10A830006C2073656E736F722034206D6F69737452
:10A840007572653A20005B20204F4B20205D20531D
:10A850006F696C2073656E736F7220332074656D41
:10A8600070657261747572653A20005B20204F4BF1
:10A8700020205D20536F696C2073656E736F7220AA
:10A8800033206D6F6973747572653A20005B202008
:10A890004F4B20205D20536F696C2073656E736F82
:10A8A0007220322074656D70657261747572653ADC
:10A8B00020005B20204F4B20205D20536F696C20CF
:10A8C00073656E736F722032206D6F697374757269
:10A8D000653A20005B20204F4B20205D20536F699C
:10A8E0006C2073656E736F7220312074656D7065B6
:10A8F0007261747572653A20005B20204F4B2020F6
:10A900005D20536F696C2073656E736F7220312008
:10A910006D6F6973747572653A20005B20204F4B30
:10A9200020205D20426174746572793A200055736D
:10A93000696E6720736F6C617220706F776572004B
:10A940002C205261773A20005573696E6720736F2F
:10A950006C61722E005761746572696E67212050B8
:10A960006C6561736520776169742E005B20204FF0
:10A970004B20205D2048756D69646974793A200028
:10A98000252C2054656D70657261747572653A206E
:10A99000005B20494E464F205D20536F696C207349
:10A9A000656E736F72203120636F6E6E65637465C0
:10A9B000642E005B20494E464F205D20536F696C2A
:10A9C0002073656E736F72203220636F6E6E6563E5
:10A9D0007465642E005B20494E464F205D20536F06
:10A9E000696C2073656E736F72203320636F6E6EB7
:10A9F00065637465642E005B20494E464F205D20E0
:10AA0000536F696C2073656E736F72203420636FAF
:10AA10006E6E65637465642E005B20494E464F2060
:10AA20005D2052756E6E696E672077617465722065
:10AA30006F6E20626F78203120666F722000207365
:10AA400065632E005B20494E464F205D2052756E97
:10AA50006E696E67207761746572206F6E20626F19
:10AA600078203220666F7220005B20494E464F20CE
:10AA70005D2052756E6E696E672077617465722015
:10AA80006F6E20626F78203320666F7220005B202B
:10AA9000494E464F205D2052756E6E696E67207775
:10AAA00061746572206F6E20626F78203420666F4B
:06AAB0007220000D0A00F7
:00000001FF
